:100000000C9412130C943A130C943A130C943A1364
:100010000C943A130C943A130C943A130C943A132C
:100020000C943A130C943A130C94B21F0C942120A4
:100030000C943A130C943A130C943A130C943A130C
:100040000C943A130C943A130C943A130C943A13FC
:100050000C943A130C943A130C943A130C945322C4
:100060000C943A130C943A130C943A130C943A13DC
:100070000C943A130C943A130C943A130C943A13CC
:100080000C943A130C943A130C943A130C943A13BC
:100090000C943A130C943A130C943A130C943A13AC
:1000A0000C943A130C943A130C943A13F0F89C8E77
:1000B0008783878E9CF8F00000FEFF030303030391
:1000C000070EFCF80000FEFF0303030303070EFC0A
:1000D000F80000FFFF00000000000000FFFF00002C
:1000E000FEFF8383838383C7EE7C380000F8FC0E19
:1000F00007030303070EFCF800003F7FE0C0808089
:10010000C0E07F3FFFFF01010101010101FFFF008E
:1001100000FFFF0C0C0C0C1C3E77E3C100007FFFBE
:10012000C0C0C0C0C0E0703F1F00001F3F70E0C0F3
:10013000C0C0E0703F1F00007FFFC1C1C1C1C1E36B
:10014000773E1C00001F3F70E0C0C0C0E0703F1F42
:10015000000000000001FFFF01000000D5F08D1439
:10016000A1C881CFD9F1AF20000B1000FCFA0676B0
:10017000567606FAFC0000F9AAABFB03FBABAAF922
:100180000000FC26AA72DE72AA26FC0000F98B8A07
:10019000FA8BFA8A8BF90000FC76DEDE26DEDE764C
:1001A000FC0000F98BFBABFBABFB8BF90000000004
:1001B00000003E5B4F5B3E3E6B4F6B3E1C3E7C3E09
:1001C0001C183C7E3C181C577D571C1C5E7F5E1C17
:1001D00000183C1800FFE7C3E7FF0018241800FFD1
:1001E000E7DBE7FF30483A060E2629792926407FCB
:1001F000050507407F05253F5A3CE73C5A7F3E1CDA
:100200001C08081C1C3E7F14227F22145F5F005FC5
:100210005F06097F017F006689956A6060606060A3
:1002200094A2FFA29408047E040810207E201008E7
:10023000082A1C08081C2A08081E101010100C1E82
:100240000C1E0C30383E3830060E3E0E0600000004
:10025000000000005F00000007000700147F147F0B
:1002600014242A7F2A122313086462364956205028
:100270000008070300001C2241000041221C002A44
:100280001C7F1C2A08083E080800807030000808FF
:10029000080808000060600020100804023E514970
:1002A000453E00427F400072494949462141494D3F
:1002B000331814127F1027454545393C4A494931C6
:1002C00041211109073649494936464949291E0045
:1002D00000140000004034000000081422411414EF
:1002E000141414004122140802015909063E415D0C
:1002F000594E7C1211127C7F494949363E41414199
:10030000227F4141413E7F494949417F0909090115
:100310003E414151737F0808087F00417F41002022
:1003200040413F017F081422417F404040407F020E
:100330001C027F7F0408107F3E4141413E7F090936
:1003400009063E4151215E7F09192946264949493E
:100350003203017F01033F4040403F1F2040201FE8
:100360003F4038403F63140814630304780403617A
:1003700059494D43007F414141020408102000418A
:1003800041417F0402010204404040404000030715
:10039000080020545478407F28444438384444446A
:1003A00028384444287F385454541800087E0902E1
:1003B00018A4A49C787F0804047800447D400020A1
:1003C00040403D007F1028440000417F40007C04F5
:1003D0007804787C080404783844444438FC1824B1
:1003E000241818242418FC7C080404084854545485
:1003F0002404043F44243C4040207C1C2040201C1A
:100400003C4030403C44281028444C9090907C4420
:1004100064544C440008364100000077000000415D
:1004200036080002010204023C2623263C1EA1A13C
:1004300061123A4040207A38545455592155557923
:1004400041215454784121555478402054557940E5
:100450000C1E527212395555555939545454593944
:10046000555454580000457C410002457D4200012E
:10047000457C40F0292429F0F0282528F07C5455AB
:1004800045002054547C547C0A097F49324949492B
:10049000323248484832324A4848303A4141217A5B
:1004A0003A42402078009DA0A07D39444444393D23
:1004B0004040403D3C24FF2424487E4943662B2F86
:1004C000FC2F2BFF0929F620C0887E0903205454F5
:1004D00079410000447D413048484A32384040224A
:1004E0007A007A0A0A727D0D19317D2629292F2872
:1004F000262929292630484D4020380808080808B0
:10050000080808382F10C8ACBA2F102834FA000099
:100510007B000008142A142222142A1408950022B1
:100520000095AA005500AAAA55AA55AA000000FFE6
:1005300000101010FF00141414FF001010FF00FF33
:100540001010F010F0141414FC001414F700FF0045
:1005500000FF00FF1414F404FC141417101F1010F3
:100560001F101F1414141F00101010F000000000C2
:100570001F101010101F10101010F010000000FFBE
:10058000101010101010101010FF10000000FF14B9
:100590000000FF00FF00001F10170000FC04F4140F
:1005A000141710171414F404F40000FF00F71414C7
:1005B0001414141414F700F7141414171410101F43
:1005C000101F141414F4141010F010F000001F1079
:1005D0001F0000001F14000000FC140000F010F0C9
:1005E0001010FF10FF141414FF141010101F00003F
:1005F0000000F010FFFFFFFFFFF0F0F0F0F0FFFF52
:10060000FF0000000000FFFF0F0F0F0F0F384444E2
:1006100038447C2A2A3E147E02020606027E027EAE
:100620000263554941633844443C04407E201E2007
:1006300006027E020299A5E7A5991C2A492A1C4CAC
:100640007201724C304A4D4D303048784830BC62AF
:100650005A463D3E494949007E0101017E2A2A2A27
:100660002A2A44445F444440514A444040444A5149
:10067000400000FF0103E080FF000008086B6B08EA
:100680003612362436060F090F060000181800002F
:10069000001010003040FF0101001F01011E001971
:1006A0001D1712003C3C3C3C0000000000101000F4
:1006B000FEFEFEDED6EAFADED6EAFAFEFEFE000016
:1006C0007F7F7B716A7B7B7B7B7B7B7B7F7F00007B
:1006D000FEFEFE5ED6EAFADED6EAFAFEFEFE000076
:1006E0007F7F6E446E6E6E6E6E6E6E6E7F7F0000EC
:1006F000FEFE7E2E6A747C6E6A747C7EFEFE0000B6
:100700007F7F5B005B5B5B5B5B5B5B5B7F7F0010AA
:100710001000FEFEFEFAEAD6DEFAEAD6DEFEFEFEA5
:1007200000007F7F7B7B7B7B7B7B7B6A717B7F7F1A
:100730000000FEFEFEFAEAD6DEFAEAD65EFEFEFE15
:1007400000007F7F6E6E6E6E6E6E6E6E446E7F7F8B
:100750000000FEFE7E7C746A6E7C746A2E7EFEFE55
:1007600000007F7F5B5B5B5B5B5B5B5B005B7F7F5A
:10077000000505000600060004000600070006004C
:10078000060004000C001C0505000700060004001C
:10079000060006001C000C0004000600062110DD07
:1007A000BAB6B6CDFFFFC0BFBFBFC0FFFF80F6F631
:1007B000F6F9FFFF80B6B6B6FFFF80F6F6F689FFC2
:1007C000FFC3BDBDDBFFC3BDBDC3FF81FBF7FB8125
:1007D000FF81B5B18FFFC3BDBDC3FFA0FFA0FFA0C8
:1007E000FF537570657220636F6D626F203D20004E
:1007F000436F6D626F203D2000506F70756C6174A7
:10080000696F6E203D2000270CFFFFC1FFC1FFC9AB
:10081000FF09FF09FFFFFFFCFC04FC04FCFCFC04D7
:10082000FC04FCFEFE02FEF2FEE2FEFEFE04FCF410
:10083000FCE4FCFCFC04FC04FC84FC94FC84FCFC58
:10084000FC84FCB4FC34FCFCFC84FCB4FC34FCFCF8
:10085000FCFFFF01FFFFFF0707040704070407046D
:10086000070407070703030607040704070407062E
:100870000707070407050704070F0F080F090F08EC
:100880000F0F0F04070407040704070407070705F1
:1008900007050704070707050705070407070707F4
:1008A00007050707070F0F00000000000000000009
:1008B0008080C0C0FF7EFFC0FF80C00080000000BD
:1008C00000000000000070207C2C7E2C7E207F2DFC
:1008D0007F2D7F217F2D7F2D7F207F2C7E2C7E20E2
:1008E0007C00700F0F00FE0676067606FE06760682
:1008F0007606FE00003F202F202F203F202F202FA4
:10090000203F0000FE82AA82AA82FEFEC6C6C6FE64
:10091000FE00003F3F3131313F3F202A202A203F57
:1009200000003CFEFE0EC6E202E2C60EFEFE3C00E9
:10093000001C3F3F202D2D202D2D203F3F1C000966
:1009400009000800D8D0F878FE3E7F78FED0F80085
:10095000D8000800000001000100000000000000B5
:1009600001000100001214000000000000008000DF
:1009700080008000E040E040FF40FF40E000E000F9
:10098000800080008000000000000000F800F800F7
:10099000F800FF07FF01FF01FF07FF01FF01FF074D
:1009A000FF01FF01FF07FF00FF00F800F800F8005B
:1009B0000F000F000F000F000F000F000F000F00BF
:1009C0000F000F000F000F000F000F000F000F00AF
:1009D0000F000F8080BFBFBFBFBFBFBFBFBFBFBFC4
:1009E000BFBFBFBFBFBFBFBFBFBFBFBFBFBF3FFF57
:1009F000FFFFFFFFFFFFFFFFFFFFFFFFFFFFFFFF07
:100A0000FFFFFFFFFFFFFFFFFFFFFFFFFFFFFFFFF6
:100A1000FFFFFFFFFFFFFFFFFFFFFFFFFFFFFFFFE6
:100A2000FFFFFFFFFFFFFFFFFFFFFFFFFFFFFFFFD6
:100A3000FFFFFFFFFFFFFFFFFFFFFFFFFFFFFFFFC6
:100A4000FFFFFFFFFFFFFFFFFFFFFFFFFFFFFFFFB6
:100A5000FFFFFFFFFFFFFFFFFFFFFFFFFFFFFFFFA6
:100A6000FFFFFFFFFFFFFFFFFFFFFFFFFFFF00FF95
:100A7000FFFFFFFFFFFFFFFFFFFFFFFFFFFFFFFF86
:100A8000FFFFFFFFFFFFFFFFFFFFFFFFFFFFFFFF76
:100A9000FFFFFFFFFFFFFFFFFFFFFFFFFFFFFFFF66
:100AA000FFFFFFFFFFFFFFFFFFFFFFFFFFFFFFFF56
:100AB000FFFFFFFFFFFFFFFFFFFFFFFFFFFFFFFF46
:100AC000FFFFFFFFFFFFFFFFFFFFFFFFFFFFFFFF36
:100AD000FFFFFFFFFFFDFD01FDFDFD01FDFDFD0130
:100AE000FDFDFD01FDFDFD01FDFDFD01FDFDFC0127
:100AF000FFFFFFFFFFFFFFFFFFFFFFFFFFFFFFFF06
:100B0000FFFFFFFFFFFFFFFFFFFFFFFFFFFFFFFFF5
:100B1000FFFFFFFFFFFFFFFFFFFFFFFFFFFFFFFFE5
:100B2000FFFFFFFFFFFFFFFFFFFFFFFFFFFFFFFFD5
:100B3000FFFFFFFFFFFFFFFFFFFFFFFFFFFFFFFFC5
:100B4000FFFFFFFFFFFFFFFFFFFFFFFFFFFFFFFFB5
:100B5000FFFFFFFFFFFEFEFEFEFEFEFEFEFEFEFEB0
:100B6000FEFEFEFEFEFEFEFEFEFEFEFEFEFEFEFEA5
:100B7000FEFEFEFE00FFFFFFFFFFFFFFFFFFFFFF88
:100B8000FFFFFFFFFFFFFFFFFFFFFFFFFFFFFFFF75
:100B9000FFFFFFFFFFFFFFFFFFFFFFFFFFFFFFFF65
:100BA000FFFFFFFFFFFFFFFFFFFFFFFFFFFFFFFF55
:100BB000FFFFFFFFFFFFFFFFFFFFFFFFFFFFFFFF45
:100BC000FFFFFFFFFFFFFFFFFFFFFFFFFFFFFFFF35
:100BD000FFFFFFFFFFFFFFFF01DDDD01DDDDDD01C9
:100BE000FFFFFFFFFFFF01DDDD01DDDDDD01FFFFB9
:100BF000FFFFFFFF00FFFFFFFFFFFFFFFFFFFFFF04
:100C0000FFFFFFFFFFFFFFFFFFFFFFFFFFFFFFFFF4
:100C1000FFFFFFFFFFFFFFFFFFFFFFFFFFFFFFFFE4
:100C2000FFFFFFFFFFFFFFFFFFFFFFFFFFFFFFFFD4
:100C3000FFFFFFFFFFFFFFFFFFFFFFFFFFFFFFFFC4
:100C4000FFFFFFFFFFFFFFFFFFFFFFFFFFFFFFFFB4
:100C5000FFFFFFFFFFFFFFFFF8FBFBF8FBFBFBF8CD
:100C6000FFFFFFFFFFFFF8FBFBF8FBFBFBF8FFFFBD
:100C7000FFFFFFFF00FFFFFFFFFFFFFFFFFFFFFF83
:100C8000FFFFFFFFFFFFFFFFFFFFFFFFFFFFFFFF74
:100C9000FFFFFFFFFFFFFFFFFFFFFFFFFFFFFFFF64
:100CA000FFFFFFFFFFFFFFFFFFFFFFFFFFFFFFFF54
:100CB000FFFFFFFFFFFFFFFFFFFFFFFFFFFFFFFF44
:100CC000FFFFFFFFFFFFFFFFFFFFFFFFFFFFFFFF34
:100CD000FFFFFFFFFFFFFFFFFFFFFFFFFFFFFF0320
:100CE000BBBB03BBBBBB03FFFFFFFFFFFFFFFFFF60
:100CF000FFFFFFFF00FFFFFFFFFFFFFFFFFFFFFF03
:100D0000FFFFFFFFFFFFFFFFFFFFFFFFFFFFFFFFF3
:100D1000FFFFFFFFFFFFFFFFFFFFFFFFFFFFFFFFE3
:100D2000FFFFFFFFFFFFFFFFFFFFFFFFFFFFFFFFD3
:100D3000FFFF07F7F7F7F7F7F7F7F7F7F7F7F7F723
:100D4000F7F7F7F7F7F7F7F7F7F7F7F707FFFFFF0B
:100D5000FFFFFFFFFFFFFFFFFFFFFFFFFFFFFFF0B2
:100D6000F7F7F0F7F7F7F0FFFFFFFFFFFFFFFFFFD9
:100D7000FFFFFFFF00FFFFFFFFFFFFFFFFFFFFFF82
:100D8000FFFFFFFFFFFFFFFFFFFFFFFFFFFFFFFF73
:100D9000FFFFFFFFFFFFFFFFFFFFFFFFFFFFFFFF63
:100DA000FFFFFFFFFFFFFFFFFFFFFFFFFFFFFFFF53
:100DB000FFFF00FFFFFFC3DBDBDBC3FFFFC3DBDBAA
:100DC000DBC3FFFFC3DBDBDBC3FFFFFF00FFFFFF76
:100DD000FFFFFFFFFFFFFF0FEFEF0FEFEFEF0FFF43
:100DE000FFFFFFFFFFFFFF0FEFEF0FEFEFEF0FFF33
:100DF000FFFFFFFF00FFFFFFFFFFFFFFFFFFFFFF02
:100E0000FFFFFFFFFFFFFFFFFFFFFFFFFFFFFFFFF2
:100E1000FFFFFFFFFFFFFFFFFFFFFFFFFFFFFFFFE2
:100E2000FFFFFFFFFFFFFFFFFFFFFFFFFFFFFFFFD2
:100E3000FFFF00FFFFFFC3DBDBDBC3FFFFC3DBDB29
:100E4000DBC3FFFFC3DBDBDBC3FFFFFF00FFFFFFF5
:100E5000FFFFFFFFFFFFFFC0DEDEC0DEDEDEC0FF04
:100E6000FFFFFFFFFFFFFFC0DEDEC0DEDEDEC0FFF4
:100E7000FFFFFFFF00FFFFFFFFFFFFFFFFFFFFFF81
:100E8000FFFFFFFFFFFFFFFFFFFFFFFFFFFFFFFF72
:100E9000FFFFFFFFFFFFFFFFFFFFFFFFFFFFFFFF62
:100EA000FFFFFFFFFFFFFFFFFFFFFFFFFFFFFFFF52
:100EB000FFFF00FFFFFFC3DBDBDBC3FFFFC3DBDBA9
:100EC000DBC3FFFFC3DBDBDBC3FFFFFF00FFFFFF75
:100ED000FFFFFFFFFFFFFFFF1FDF5F5F5F5F5F5FE2
:100EE0005F5F5F5F5F5F5F5F5F5FDF1FFFFFFFFF52
:100EF000FFFFFFFF00FFFFFFFFFFFFFFFFFFFFFF01
:100F0000FFFFFFFFFFFFFFFFFFFFFFFFFFFFFFFFF1
:100F1000FFFFFFFFFFFFFFFFFFFFFFFFFFFFFFFFE1
:100F2000FFFFFFFFFFFFFFFFFFFFFFFFFFFFFFFFD1
:100F3000FFFF00FFFFFFC3DBDBDBC3FFFFC3DBDB28
:100F4000DBC3FFFFC3DBDBDBC3FFFFFF00FFFFFFF4
:100F5000FFFFFFFFFFFFFFFF00FF00FFFF03FBFBA3
:100F6000FBFB03FBFBFB03FFFF00FF00FFFFFFFF9B
:100F7000FFFFFFFF00FFFFFFFFFFFFFFFFFFFFFF80
:100F8000FFFFFFFFFFFFFFFFFFFFFFFFFFFFFFFF71
:100F9000FFFFFFFFFFFFFFFFFFFFFFFFFFFFFFFF61
:100FA000FFFFFFFFFFFFFFFFFFFFFFFFFFFFFFFF51
:100FB000FFFF00FFFFFFFFFFFFFFFF0FEFEFEF0F50
:100FC000EFEFEF0FFFFFFFFFFFFFFFFF00FFFFFF50
:100FD000FFFFFFFFFFEFEFEFE0EFE0EFEFE0EFEFFE
:100FE000EFEEE0EFEFEFE0EFEFE0EFE0EFEFEFEF4E
:100FF000EFEFEFEFE0EFEFEFEFEFEFEFEFEFEFEF10
:10100000EFEFEFEFEFEFEFEFEFEFEFEFEFEFEFEFF0
:10101000EFEFEFEFEFEFEFEFEFEFEFEFEFEFEFEFE0
:10102000EFEFEFEFEFEFEFEFEFEFEFEFEFEFEFEFD0
:10103000EFEFE0EFEFEFEFEFEFEFEFE0EFEFEDE0EF
:10104000EDEFEFE0EFEFEFEFEFEFEFEFE0EFEFEFD0
:10105000EFEFEFEFEFFFFFFFFFFFFFFFFFFFFFFFF0
:10106000FFEFFFFFFFFFFFFFFFFFFFFFFFFFFFFFA0
:10107000FFFF7F0FA1A4A10F7FFFFFFFFFFFFFFF77
:10108000FFFF3FDFDFDDDFDFDFDFDFDFDFDFDFDFD2
:10109000DFDFDFDFDFDFDFDFDFDFDFDFDFDFDFDF60
:1010A000DFDFDFDFDFDFDFDFD7DF3FFFFFFFFFFF58
:1010B000FFFFFF7F0FA1A4A10F7FFFFFFFFFFFFF37
:1010C000FFFFFFFFFFFFFFFFFFFFFFFFFBFFFFFF34
:1010D000FFFFFFFFFFFFFFFFDFFFFFFFFFFFFFFF40
:1010E000FFFFFFFFFFFFFFFFFFFFFBFFFF7F0F275C
:1010F0000F7FFEFEFEFEFEFEFEFFFFFFFFFF3FCF67
:10110000F3FCFFFFFFFFFFFFFFFFFFFFFFFFFFFFFE
:10111000FFFFFFFFFFFFFFFFFFFFFFFFFFFFFFFFDF
:10112000FFFFFFFFFFFFFFFFFFFFFFFCF3CF3FFFCE
:10113000FFFFFFFEFEFEFEFEFEFE7F0F270F7FFF7E
:10114000FFFFFFFFFFFFFFFFFFFFFFFFFFFFF7FFB7
:10115000FFFFFFFFFFFFFFFFFFFFFFFFFFFFFFFF9F
:10116000FFF7FFFFFFFFFFFFFFFFFFFFF3F0F5F5C6
:10117000F5F0F3FFFFFFFFFFFFFF3FCFF3FCFFFFA3
:10118000FFFFFFFFFFFFFFFFFFFFFFFFFFFFFFFF6F
:10119000FFFFFFFFFFFFFFFFFFFFFFFFFFFFFFFF5F
:1011A000FFFFFFFFFFFFFFFFFFFFFFFFFFFFFFFC52
:1011B000F3CF3FFFFFFFFFFFFFF3F0F5F5F5F0F38F
:1011C000FFFFFFFFFFFFBFFFFFFFFFFFFFFFFFFF6F
:1011D000FFFFFFFFFF8040FFFFFFFFFFFFFFFFFF5D
:1011E000FFFFFFFFFFFFFFFFFFFFFFFFFFFFFFFF0F
:1011F000FFFFFFFFFFFFFFFFFFFFFFFFFFFFFFFFFF
:10120000FFFFFFFFFFFFBFFFFFFFFFFFFFFFFFFF2E
:10121000FFFFFFFFFFFFFFFFFFFFFFFFFFFFFFFFDE
:10122000FFFFFFFFFFFFFFFFFFFFFFFFFFFFFFFFCE
:10123000FFFFFFFFFFFFFFFFFFFFFFFFFFFFFFFFBE
:10124000FFFFFFFFFFFFFFFFFFFFFFFFFFFFFFFFAE
:10125000FFFFFFFFFFFFFFFFFFFFFFFFFFFFFFFF9E
:10126000FFFFFFFFFFFFFFFFFF7F3F7FFFFFFFFF4E
:10127000FFFFFFFFFFFFFFFFFFFFFFFFFFFFFFFF7E
:10128000FFFFFFFFFFFFFFFFFFFFFFFFFFFFFFFF6E
:10129000FFFFFFFFFFFFFFFFFFFFFFFFFFFFFFFF5E
:1012A000FFFFFFFFFFFFFFFFFFFFFFFFFFFFFFFF4E
:1012B000FFFFFFFFFFFFFFFFFFFFFFFFFBFFFFFF42
:1012C000FFFFFFFFFFFFFFFFFFFFFFFFFFFFFFFF2E
:1012D000FFFFFFFFFFFFFFFFFFFFFFFFFFFFFFFF1E
:1012E000FFFFFFFFFFFFFFFFFEFCF8FCFEFFFFFF1D
:1012F000FFFFFFFFFFFFFFFFFFFFFF7F1FCFEFEFAE
:10130000E7E389FDFDFDFDFDFDFDFDF9F3C79F3F11
:10131000FFFFFFFFFFFFFFFFFFFFFFFFFFFFFFFFDD
:10132000FFFFFFFFFFFFFFFFFFFFFFFFFFFFFFFFCD
:10133000FFFFFFFFFFFFFFFFFFFFFFFFFFFFFFFFBD
:10134000FFFFFFFFFFFFFFFFFFFFFFFFFFFFFFFFAD
:10135000FFFFFFFFFFFFFFFFFFFFFFFFFFFFFFFF9D
:10136000FFFFFFFFFFFFFFFFFFFFFFFFFFFFFFFF8D
:10137000FFFFFFFFFFFFFFFFFFFFFFFCFDF9FBFB90
:10138000FBFBFBFBFBF9FDFCF9FBFBFBFBF9FDFCAD
:10139000FFFFFFFFFFFFFFFFFFFFFFFFFFFFFFFF5D
:1013A000FFFFFFFFFFFFFFFFFFFFFFFFFFFFFFFF4D
:1013B000FFFFFFFFFFFFFFFFFFFFFFFFFFFFFFFF3D
:1013C000FFFFFFFFFFFFFFFFFFFFFFFFFFFFFFFF2D
:1013D000FFFFFFFFFFFFFFFFFFFFFFFFFFFFFFFF1D
:1013E000FFFFFFFFFFFFFFFFFFFFFFFFFFFFFFFF0D
:1013F000FFFFFFFFFFFFFFFFFFFFFFFFFFFFFFFFFD
:10140000FFFFFFFFFFFFFFFFFFFFFFFFFFFFFFFFEC
:10141000FFFFFFFFFFFFFFFFFFFFFFFFFFFFFFFFDC
:10142000FFFFFFFFFFFFFFFFFFFFFFFFFFFFFFFFCC
:10143000FFFFFFFFFFFFFFFFFFFFFFFFFFFFFFFFBC
:10144000FFFFFFFFFFFFFFFFFFFFFFFFFFFFFFFFAC
:10145000FFFFFFFFFFFFFFFFFFFFFFFFFFFFFFFF9C
:10146000FFFFFFFFFFFFFFFFFFFFFFFFFFFFFFFF8C
:10147000FFFFFFFFFFFFFFFFFFFFFFFFFFFFFFFF7C
:10148000FFFFFFFFFFFFFFFFFFFFFFFFFFFFFFFF6C
:10149000FFFFFFFFFFFFFFFFFFFFFFFFFFFFFFFF5C
:1014A000FFFFFFFFFFFFFFFFFFFF7FFFFFFFFFFFCC
:1014B000FFFFFFFFFFFFFFFFFFFFFFFFFFFFFFFF3C
:1014C000FF3FCFE7F7F7F7F3C39BFDFDFDF9FBFB0C
:1014D000F3C7DFDFBF3FFFFFFFFFFFFFFFFFFFFFA0
:1014E000FFFFFFFFFFFFFFFFFFFFFFFFFFFFFDFF0E
:1014F000FFFFFFFFFFFFFFFFFFFFFFFFFFFFFFFFFC
:10150000FFFFFFFFFFFFFFFFFFFFFFFFFFFFFFFFEB
:10151000FFFFFFFFFFFFFFFFFFFFFFFFFFFFFFFFDB
:10152000FFFFFFFFFFFFFFFFFFFFFFFFFFFFFFFFCB
:10153000FFFFFFFFFFFFFFFFFFFFFFFFFFFFFFFFBB
:10154000FFFEFDF9FBFBF3F7F7F3FBFBF9F9FBFB00
:10155000F7F7F7F3F9FCFFFFFFFFFFFFFFFFFFFFC8
:10156000FFFFFFFFFFFFFFFFFFFFFFFFFFFFFFFF8B
:10157000FFFFFFFFFFFFFFFFFFFFFFFFFFFFFFFF7B
:10158000FFFFFFFFFFFFFFFFFFFFFFFFFFFFFFFF6B
:10159000FFFFFFFFFFFFFFFFFFFFFFFFFFFFFFFF5B
:1015A000FFFFFFFFFFFFFFFFFFFFFFFFFFFFFFFF4B
:1015B000FFFFFFFFFFFFFFFFFFFFFFFFFFFFFFFF3B
:1015C000FFFFFFFFFFFFFFFFFFFFFFFFFFFFFFFF2B
:1015D000FFFFFFFFFFFFFFFFFFFFFFFFFFFFFFFF1B
:1015E000FFFFFFFFFFFFFFFFFFFFFFFFFFFFFFFF0B
:1015F000FFFFFFFFFFFFFFFFFFFFFFFFFFFFFFFFFB
:10160000FFFFFFFFFFFFBFFFFFFFFFFFFFFFFFFF2A
:10161000FFFFFFFFFFFFFFFFFFFFFFFFFFFFFFFFDA
:10162000FFFFFFFFFFFFFFFFFFFFFFFFFFFFFFFFCA
:10163000FFFFFFFFFFFFFFFFFFFFFFFFFFFFFFFFBA
:10164000FFFFFFFFFFFFFFFFFFFFFFFFFFFFFFFFAA
:10165000FFFFFFFFFFFFFFFFFFFFFFFFFFFFFFFF9A
:10166000FFFFFFFFFF7F7F7F7FFFFFFFFFFFFFFF8A
:10167000FFFFFFFFFFFFFFFFFFFFFFFFFFFFFFFF7A
:10168000FFFFFFFFFFFFFFFFFFFFFFFFFFFFFFFF6A
:10169000FFFFFFFFFFFFFFFFFFFFFFFFFFFFFFFF5A
:1016A000FFFFFFFFFFFFFFFFFFFFFFFFFFFFFFFF4A
:1016B000FFFFFFFFFFFFFFFFFFFFFFFFFBFFFFFF3E
:1016C000FFFFFFFFFFFFFFFFFFFFFFFFFFFFFFFF2A
:1016D000FFFFFFFFFFFFFFFFFFFFFFFF8F7379FD9E
:1016E000FDFDFCF0E6FFFF7F7EFEFEFCF1F7F76FED
:1016F0000FFFFFFFFFFFFFFFFFFFFFFFFFFFFFFFEA
:10170000FFFFFFFFFFFFFFFFFFFFFFFFFFFFFFFFE9
:10171000FFFFFFFFFFFFFFFFFFFFFFFFFFFFFFFFD9
:10172000FFFFFFFFFFFFFFFFFFFFFFFFFFFFFFFFC9
:10173000FFFFFFFFFFFFFFFFFFFFFFFFFFFFFFFFB9
:10174000FFFFFFFFFFFFFFFFFFFFFFFFFFFFFFFFA9
:10175000FFFFFFFFFFFFFFFFFFFFFFFFFFFFFEFE9B
:10176000FEFCFDFDFCFEFEFEFEFEFEFDFDFDFCFEA4
:10177000FFFFFFFFFFFFFFFFFFFFFFFFFFFFFFFF79
:10178000FFFFFFFFFFFFFFFFFFFFFFFFFFFFFFFF69
:10179000FFFFFFFFFFFFFFFFFFFFFFFFFFFFFFFF59
:1017A000FFFFFFFFFFFFFFFFFFFFFFFFFFFFFFFF49
:1017B000FFFFFFFFFFFFFFFFFFFFFFFFFFFFFFFF39
:1017C000FFFFFFFFFFFFFFFFFFFFFFFFFFFFFFFF29
:1017D000FFFFFFFFFFFFFFFFFFFFFFFFFFFFFFFF19
:1017E000FFFFFFFFFFFFFFFFFFFFFFFFFFFFFFFF09
:1017F000FFFFFFFFFFFFFFFFFFFFFFFFFFFFFFFFF9
:10180000FFFFFFFFFFFFFFFFFFFFFBF1E0F1FBFF2B
:10181000FFFFFFFFFFFFFFFFFFFFFFFFFFFFFFFFD8
:10182000FFFFFFFFFFFFFFFFFFFFFFFFFFFFFFFFC8
:10183000FFFFFFFFFFFFFFFFFFFF7F3F9FDFDFDFB8
:10184000DFDFDFDFDF9F3F7FFFFFFFFFFFFFFFFFE8
:10185000FFFFFFFFFFFFFFFFFFFFFFFFFFFFFFFF98
:10186000FFFFFFFFFFFFFFFFFFFFFFFFFFFFFFFF88
:10187000FFFFFFFFFFFFFFFFFFFFFFFFFFFFFFFF78
:10188000FFFFFFFFFFFFFFFFFFFFFFFFFFFFFFFF68
:10189000FFFFFFFFFFFFFFFFFFFFFFFFFFFFFFFF58
:1018A000FFFFFFFFFFFFFFFFFFFF7FFFFFFFFFFFC8
:1018B000FFFFFFFFFFC7D19CBEBEBEBEB8BFBF9F2C
:1018C000DFCF9FBFBFBFBF9CD9C3FFFFFFFFFFFF9D
:1018D000FFFFFFFFFFFFFFFFFFFFFFFFFFFFFFFF18
:1018E000FFFFFFFFFFFFFFFFFFFFFFFFFFFFFDFF0A
:1018F000FFFFFFFFFFFFFFFFFFFFFFFFFFFFFFFFF8
:10190000FFFFFFFFFFFFFFFFFFFFFFFFFFFFFFFFE7
:10191000FFFFFFFFFFFFFFFFFFFFFFFFFFFFFFFFD7
:10192000FFFFFFFFFFFFFFFFFFFFFFFFFFFFFFFFC7
:10193000FFFFFFFFFFFFFFFFFFFFFFFFFFFFFFFFB7
:10194000FFFFFFFFFFFFFFFFFFFFFFFFFFFFFFFFA7
:10195000FFFFFFFFFFFFFFFFFFFFFFFFFFFFFFFF97
:10196000FFFFFFFFFFFFFFFFFFFFFFFFFFFFFFFF87
:10197000FFFFFFFFFFFFFFFFFFFFFFFFFFFFFFFF77
:10198000FFFFFFFFFFFFFFFFFFFFFFFFFFFFFFFF67
:10199000FFFFFFFFFFFFFFFFFFFFFFFFFFFFFFFF57
:1019A000FFFFFFFFFFFFFFFFFFFFFFFFFFFFFFFF47
:1019B000FFFFFFFFFFFFFFFFFFFFFFFFFFFFFFFF37
:1019C000FFFFFFFFFFFFFFFFFFFFFFFFFFFFFFFF27
:1019D000FFFFFFFFFFFFFF534B5953434541504566
:1019E00052210061206E6577206275696C64696EB2
:1019F000673A00596F752068617665206F70656E73
:101A0000656400544F57455220424C4F434B2100D0
:101A100061206E6577206275696C64696E673A0053
:101A2000596F752068617665206F70656E6564001A
:101A30006F66206275696C64696E67007468652002
:101A4000666972737420747970650070726F76695C
:101A500064656420796F75207769746800596F75C3
:101A60007220696E766573746F72206861730069A5
:101A70006E746F2061206D656761706F6C697300B3
:101A80007475726E207468697320746F776E006F5E
:101A900066206C616E642E20596F75206D617374C1
:101AA00000596F75206861766520612070696563F3
:101AB000650041524455424C4F5858210057656CBF
:101AC000636F6D6520746F004D656761706F6C6941
:101AD00073004D617374657200476F6C64656E20AE
:101AE0006275696C64696E67004561676C65206545
:101AF0007965001414FF0101110901012171F9ED4B
:101B0000F9F1E1E181010101FFFF000080C0E07017
:101B1000381C0E0703070F1F8D070200FF0F080B6D
:101B20000B09080808080808080808090808080830
:101B30000FFF0101F19151FD250595FD1151F12195
:101B4000A1E10101FFFF00FC1584FC8180F8282938
:101B50008888F9404041C000FF0F080B08080B08B7
:101B6000080B080808080B0808090B080FFF0101FB
:101B70004101010181413D3D418101010109010115
:101B8000FFFF0000F8080E5A4B5A0B0B5A4B5A0E27
:101B900008F80000FF0F08080F08080A0A0A0808DA
:101BA0000A0A0A08080F08080FFF030509914121D6
:101BB000A161212161A1214191090503FFFF000ECF
:101BC0001120409FA0C08686C0A09F4020110E001B
:101BD000FF0F0C0A09080808080808080808080880
:101BE00008090A0C0F416368696576656D656E7456
:101BF0007300636F6D706C657465642100436F6E74
:101C0000737472756374696F6E00436F6E6772618F
:101C100074756C6174696F6E732100616E79776899
:101C20006572652E005075742061206E657720689E
:101C30006F6D6500757020612063697479003133C0
:101C4000206461797320746F206275696C6400523E
:101C5000656D656D62657220796F75206861766566
:101C600000536B797363726170657200353600548E
:101C70006F77657220626C6F636B003337004D6164
:101C800069736F6E6574746500323400140900FC6A
:101C9000AAF9AAFC000000000000000000000000FB
:101CA0000000000000000000000000000000000034
:101CB00000000000000019090000AE7EAE00000028
:101CC0000000000000000000000000000000000014
:101CD0000000000000000000000000000000000004
:101CE00000000000000000000000101000FCFAF6E8
:101CF0000EEE6EAEAE6EEE0EF6FAFC00003F5F6FBB
:101D000070777675757677706F5F3F0000FC86BAE6
:101D1000BAFAA27E7EA2FABABA86FC00003F615DE2
:101D20005D5F457E7E455F5D5D613F0000FCFE5668
:101D30006E563E86863E566E56FEFC00003F7F6A1B
:101D4000766A7C61617C6A766A7F3F00422D71759C
:101D50006974006661696C656400436F6E737472C8
:101D6000756374696F6E00422D7175697400412D41
:101D7000737461790077696C6C206265206C6F7395
:101D80007400796F75722070726F6772657373007B
:101D9000496620796F7520717569740050415553FB
:101DA00045008040FF8000000000000000000000AF
:101DB0000000000000000000000000000000000023
:101DC00000000000FF0000573F5700000000000027
:101DD0000000000000000000000000000000000003
:101DE000000000000000000000000000FF000F09DC
:101DF000392F243C0000000000000000000000001B
:101E00000000000000000010101054381000000006
:101E100000000000000000000000000000000000C2
:101E2000000080FFFFFE06E6F6F6F6F6F6F6F6F69A
:101E3000F6F6F6F6E606FEFE7E3E9ECEE6F6F67672
:101E400076767676777676767676F6F6F6F6F6F631
:101E5000F6F6F6F6F6F6F6F6767676767676767622
:101E6000767676F6F6F606F6F696F6F607F6F6F6D1
:101E7000F67676767676767676767676F6F6F6F682
:101E8000F6F6F6F6F6F6B6F6F6F676767676767632
:101E90007676767676F6F6F6F6F6E6CE9E3E7EFE1A
:101EA000FEFEFEFFFFFF00FFFFFFFFFFFFFFFFFF44
:101EB000FFFFFFFFFF00FF00FEFFFFFFFFFFFF0030
:101EC000FFFFFFFFFFFFFFFFFF00FFFFFFFFFFFF21
:101ED000FFFFFFFFFEFFFFFF00FFFFFFFFFFFFFF12
:101EE000FFFF00FFFFFF00FFFF33FFFF00FFFFFFCB
:101EF000FF00FFFFFFFFFFFFFFFFFF00FFFFFFFFF0
:101F00007FFFFFFFFFFFFFFFFFFF00FFFFFFFFFF60
:101F1000FFFFFFFF00FFFFFFFFFFFFFFFFFFFE00D0
:101F2000FFFFFFFFFFFF08C9EBEBEBEBEBEBEBEB8E
:101F3000EBEBEBEBC908FF007F7F7F7F6F7F7F7C40
:101F40007D7D7D7D7D7D7D7D7D7C7F7F7F7F7F7FB6
:101F50006F7F7F7F7F7F7F7F7C7D7D7D7D7D7D7DB2
:101F60007D7D7C7FBFDFE0FFFFE7FFFFE0DFBF7F1E
:101F70007F7C7D7D7D7D7D7D7D7D7D7C7F7F7F7E8A
:101F8000717A7F7F7F7F7F7B7F7F7C7D7D7D7D7D85
:101F90007D7D7D7D7C7F7F7F7F7F7F6F7F7F7F00EB
:101FA000FFFFFFFFFFFF00FFFFFFFFFFFFFFFFFF40
:101FB000FFFFFFFFFF00FF00777777777F7F7F7F4F
:101FC0007F7F777777777F7F7F7F7F7F7777777761
:101FD0007F7F7F7F7F7F777777777F7F7F7F7F7F31
:101FE0007F777777F7FFFFFFFFFFFFFFFFFFF777B1
:101FF00077777F7F7F7F7F7F777777777F7F7F7F21
:102000007F7F777777777F7F7F7F7F7F7F77777718
:10201000777F7F7F7F7F7F777777777F7F7F7F0077
:10202000FFFFFFFFFFFF1093D7D7D7D7D7D7D7D75B
:10203000D7D7D7D79310FF00FFFFFFFFFFFFFF1F8A
:10204000DFDFDFDFDFDFDFDFDF1FFFFFFFFFFF7F20
:10205000FFFFFFFFFFFFFFFF1FDFDFDFDFDFDFDF50
:10206000DFDF1FFFFEFD03FFFF73FFFF03FDFEFF2A
:10207000FF1FDFDFDFDFDFDFDFDFDF1FFFFFFFF758
:10208000FFFFFFFFFFFFFFFFFFFF1FDFDFDFDFDFE0
:10209000DFDFDFDF1FFFFFFFFFFFFFFFFFFFFF00AF
:1020A000FFFFFFFFFFFF00FFFFFFFFFFFFFFFFFF3F
:1020B000FFFFFFFFFF00FF007FFFFEFFFFFFFF00AE
:1020C0007F7F7F7F7F7F7F7F7F00FFFFEF17AFFFE7
:1020D000FFFFFFFFFFFFFFFF007F7F7F7F7F7F7F8F
:1020E0007F7F00FFFFFF00FFFFE6FFFF00FFFFFF16
:1020F000FF007F7F7F7F7F7F7F7F7F00FFFFFFFF6E
:10210000FFFFFFFFFFEFFFFFFFFF007F7F7F7F7F6E
:102110007F7F7F7F00FFFFFFFFFFFFFFFDFF7F004F
:10212000FFFFFFFFFFFFE0E7EFEFEFEFEFEFEFEF76
:10213000EFEFEFEFE7E0FFFFFEFCF9F3E7EFEFEF84
:10214000EFEFEFEFEFEFEFEFEFEFEFEFEFEFEFEF9F
:10215000EFEFEFEFEFEFEFEFEFEFEFEFEFEFEFEF8F
:10216000EFEFEFEFEFEFE0EFEFECEFEFE0EFEFEFA0
:10217000EFEFEFEFEFEFEFEFEFEFEFEFEFEFEFEF6F
:10218000EFEFEFEFEFEFEFEFEFEFEFEFEFEFEFEF5F
:10219000EFEFEFEFEFEFEFEFEFEFE7F3F9FCFEFF1D
:1021A000FFFFFFFF0505100A070E04804000000036
:1021B0000000000000FC0404040484C4E47434340B
:1021C00074E4C484040404F4949494F4F48404043F
:1021D0000404F4F4343474E4C40404F4F40404048F
:1021E00004F4F404040404040404040404040404CF
:1021F000F4949494F4F4040404F4F404040404043F
:1022000004C4E47434343474E4C404043464C4840E
:102210000484C464340404043464C4840484C4643E
:1022200034040404FC000000000000000000000072
:102230000000000000FF80808080BFBF8484848411
:102240008484BFBF808080BFBF81818181BFBF8008
:102250008080BFBFB0B0B89F8F80809FBFB0B0B04C
:10226000B0BF9F80808080808787878080808080CB
:10227000BFA1A1A1A1BFBF8080BFBFB0B0B8B880CF
:10228000808F9FB8B0B0B0B89F8F8080B0988C8797
:1022900083878C98B0808080B0988C8783878C9857
:1022A000B0808080FF0000000000000000000000FF
:1022B000000000000000000000000000000000001E
:1022C000000000000000000000000000000000000E
:1022D00000000000000000000000000000000000FE
:1022E00000000000000000000000000000000000EE
:1022F00000000000000000000000000000000000DE
:1023000000000000000000000000000000000000CD
:1023100000000000000000000000000000000000BD
:1023200000000000000000000000000000000000AD
:10233000000000000000000000000000000000009D
:1023400000000000000000000000FF01FD95FD01FD
:10235000FD95FD01FF0000000000000000000000EE
:10236000000000000000000000000000000000006D
:10237000000000000000000000000000000000005D
:10238000000000000000000000000000000000004D
:10239000000000000000000000000000000000003D
:1023A000000000000000000000000000000000002D
:1023B0000000000000008040209048E4C8902040C9
:1023C0008000000000FC04F454F407F656F606FE04
:1023D00002020202030000000000000000000000F2
:1023E00000000000000000000000000000000017D6
:1023F000151D00011F01001E051E001F0507180105
:102400001F010000001E051E000000001F1111002A
:102410001F111F001F0204021F001F0507001E05D9
:102420001E001F02041F00031C0300000000000028
:1024300000000000000102040913274E25130904BF
:1024400002010000000F080B0A0B08FB0AEBA8EFC3
:1024500008E8A8E808F800000000000000000000FC
:10246000000000000000C0603018080808080808D4
:1024700008183060C00000000000000000000000EC
:10248000000000000000000000000000000000004C
:10249000000000000000002E2A3A003828380038DA
:1024A0002038003808380038283C000000000000C0
:1024B000000000000000000000000000000000001C
:1024C0000000000000000000F010D05FD017D457CB
:1024D000D017F417101F00000000000000000000DB
:1024E000E0E060408000037E8202025AC2C2C25A0B
:1024F0000202827E0300804060E0E00000000000F5
:1025000000000000000000000000000000000000CB
:1025100000000000000000000000000000000000BB
:1025200000000000000000000000000000000000AB
:10253000000000000000000000000000000000009B
:1025400000000000000000003F202F292F202F292D
:102550002F203F00000000000000000000000000ED
:1025600000010204081122C40465660A1222120A3C
:10257000060504C422110804020100000000000046
:10258000000000000000000000000000000000004B
:10259000000000000000000000000000000000003B
:1025A00000000000000000000000000000080B0018
:1025B00002020200000904000001020200000524DA
:1025C000001001052401010104240206052406006F
:1025D000010705810310004009040100020A000000
:1025E00000070502024000000705830240000004C6
:1025F00003090412010002EF02014041233680006A
:10260000010102030141726475696E6F204C4C43F5
:102610000041726475696E6F204C656F6E61726403
:102620006F00D02211241FBECFEFDAE0DEBFCDBF96
:1026300011E0A0E0B1E0ECE4FFE602C005900D92ED
:10264000A038B107D9F726E0A0E8B1E001C01D929B
:10265000AE33B207E1F713E1C2E1D3E104C0219741
:10266000FE010E949E37C131D107C9F70E94ED22B9
:102670000C94A4370C940000EAEEF1E0A0E0B8E07E
:1026800000800EBC8111012C1197A0FDFDCF01929D
:10269000B9F70DB40895FC018091E901882311F187
:1026A0003FB7F89482E08093E9002091F200822FF6
:1026B00090E01816190614F481E090E0882339F0B0
:1026C000289844E64093E8014091F100408322239A
:1026D00039F02091F200211103C02BE62093E8008D
:1026E0003FBF08958FEF9FEF08952FB7F89483E0D1
:1026F0008093E9009091E800892F807295FF04C0D3
:102700009091F20080E4891B2FBF08958091E00131
:1027100081110DC082E08093DC0184E08093DD01B3
:102720001092DF011092DE0181E08093E0018CEDD8
:1027300091E00895CF93DF931F92CDB7DEB7698301
:10274000DC01ED91FC910280F381E02D41E050E04D
:10275000BE016F5F7F4F09950F90DF91CF91089574
:1027600083E08093E9008091F200882319F08AE3E6
:102770008093E80008950E94751390E00895CF9328
:10278000DF931F92CDB7DEB7FC018485958597FD59
:1027900008C02FEF3FEF358724870F90DF91CF914F
:1027A0000895CE0101960E944B13019719F4898177
:1027B00090E0F3CF8FEF9FEFF0CF0F931F93CF9366
:1027C000DF931F92CDB7DEB78C01FC018485958520
:1027D00097FF0BC0CE0101960E944B13019771F435
:1027E000898190E0F80195878487F8018485958533
:1027F0000F90DF91CF911F910F9108958FEF9FEF71
:10280000F1CFFC018485958597FD0BC09FB7F894A7
:1028100082E08093E9008091F2009FBF90E00196F2
:1028200008959FB7F89482E08093E9008091F200C8
:102830009FBF90E008954091D6015091D70120911B
:10284000D4013091D50142175307B4F49091E800B8
:102850009570E1F39091E80092FD19C08093F1002A
:102860008091D6019091D70101968F739927892B7A
:1028700019F48EEF8093E8008091D6019091D701F2
:1028800001969093D7018093D60181E0089580E06E
:102890000895DF92EF92FF920F931F93CF93DF93F0
:1028A000D82E8A01EB017B01E40EF51ECE15DF0563
:1028B00059F0D7FE12C0FE0184910E941B1421968C
:1028C0008111F4CF0FEF1FEFC801DF91CF911F915E
:1028D0000F91FF90EF90DF9008958881EECF0F93D6
:1028E0001F93CF93DF931F92CDB7DEB782E089832A
:1028F00042E450E06DEA75E280E80E9449140E94CB
:102900008613DC0112960D911C910115110589F0B9
:10291000D801ED91FC910280F381E02DBE016F5F43
:102920007F4FC801099597FD04C0F8010085118506
:10293000ECCF89810F90DF91CF911F910F91089576
:10294000615030F02091F100FC0120830196F8CF16
:10295000289884E68093E8010895AF92BF92CF92C1
:10296000DF92EF92FF920F931F93CF93DF936C014F
:102970007B018B01040F151FEB015E01AE18BF0830
:10298000C017D10759F06991D601ED91FC910190E2
:10299000F081E02DC6010995892B79F7C501DF91FA
:1029A000CF911F910F91FF90EF90DF90CF90BF904C
:1029B000AF9008953FB7F8948091890190918A0172
:1029C000A0918B01B0918C0126B5A89B05C02F3F2B
:1029D00019F00196A11DB11D3FBFBA2FA92F982F45
:1029E0008827BC01CD01620F711D811D911D42E040
:1029F000660F771F881F991F4A95D1F708958F9208
:102A00009F92AF92BF92CF92DF92EF92FF926B01B3
:102A10007C010E94DA144B015C01C114D104E10471
:102A2000F104B9F00E94DA14681979098A099B093E
:102A3000683E73408105910580F321E0C21AD108F8
:102A4000E108F10888EE880E83E0981EA11CB11CF5
:102A5000E4CFFF90EF90DF90CF90BF90AF909F902A
:102A60008F9008958F929F92AF92BF92CF92DF92F4
:102A7000EF92FF920F931F93CF93DF936C017B0133
:102A80008A0180913501882309F45CC08091E901B5
:102A9000882309F457C08091DB0180FF05C0809135
:102AA000E00082608093E000E801B12C8AEFA82E5C
:102AB00093E0892E2AE3922E209711F4BB20D9F1BE
:102AC0000E94751381110AC0AA94AA20D9F161E06D
:102AD00070E080E090E00E94FF14EECF8C171D069E
:102AE00011F00CF08C2F9FB7F8948092E9002091A0
:102AF000E80025FD02C09FBFDFCF282F30E0C21BBA
:102B0000D30BF701815020F041914093F100FACFAF
:102B1000E20EF31EBB2021F09092E800B12CEBCF27
:102B20008091E80085FDE7CF9092E800BB24B39444
:102B3000209709F3F3CF5D9884E68093DA011016AD
:102B400011063CF081E090E0F6019383828310E06F
:102B500000E0C801DF91CF911F910F91FF90EF909E
:102B6000DF90CF90BF90AF909F908F9008954F923D
:102B70005F926F927F928F929F92AF92BF92CF920D
:102B8000DF92EF92FF920F931F93CF93DF934C014D
:102B90005901FC2DC02FD0E0CE01880D991D1816CB
:102BA00019060CF06CC020E8821691040CF067C086
:102BB0009B012E0D311D121613060CF060C06034FF
:102BC00071050CF05CC04115510509F458C0E62FA1
:102BD000E770FE2EDB0177FD179633E0B595A795DC
:102BE0003A95E1F73A2F77FF04C0FF2011F03FEF4D
:102BF0003A0F662777276819790997FC02C070E0B9
:102C000060E0803891050CF44BC090E89819961B51
:102C1000A32F032E000CBB0B1A2F10953F3F0CF077
:102C200010E021E08E2D877009F420E0E694E69410
:102C3000E694E20EAE0DB11D19971CF028E0E22ECD
:102C4000E31AE11A310F20E83203D0011124A80D54
:102C5000B91DA60FB71F019F600D711D1124460FEE
:102C6000571F0F2D0F2C000C110BF33009F41CC152
:102C7000C8F4F13009F4D0C0F23009F47CC0DF911F
:102C8000CF911F910F91FF90EF90DF90CF90BF9069
:102C9000AF909F908F907F906F905F904F9008952E
:102CA000902FB5CFFA3FB1F1232F2E0DFB3F39F70F
:102CB000321729F3BD0166517E4FD12CC12CC916A4
:102CC00008F0A4C0FA01EC0DFD1DE491F0E04F0105
:102CD000002E02C0880C991C0A94E2F737FD06C04A
:102CE000FB018081E82CE0948E218083FF2061F03D
:102CF000373054F45B01F0E8AF0EB11CE92CE094DE
:102D0000F50180818E218083FFEFCF1ADF0A6F5F8C
:102D10007F4FD5CF232F2E0D321709F4B0CFBD0131
:102D200066517E4FD12CC12CC91608F069C0FA013A
:102D3000EC0DFD1DE491F0E04F01002E02C0880C67
:102D4000991C0A94E2F737FD04C0FB0180818829B1
:102D50008083FF2051F0373044F45B01F0E8AF0E80
:102D6000B11CF501808189298083FFEFCF1ADF0A2A
:102D70006F5F7F4FD9CF6FEF70E00F2C02C0660FEF
:102D8000771F0A94E2F760957095772E232F2E0D0A
:102D9000321709F474CFFD01E651FE4F6F01B12CDB
:102DA000A12CA91638F5FA01EA0DFB1DE491F0E01B
:102DB0002F01002E02C0440C551C0A94E2F737FD87
:102DC00005C0F6018081862384298083FF2059F085
:102DD00037304CF44601F0E88F0E911CF4018081ED
:102DE000872185298083FFEFAF1ABF0A8FEFC81AAA
:102DF000D80AD7CF3F5F4C0F5D1FA058BF4FC8CF39
:102E00003F5F4C0F5D1FA058BF4F86CF3F5F4C0FF9
:102E10005D1FA058BF4F4CCF6A0D7B1D232F2E0D79
:102E2000321709F42CCFFD01E651FE4F6F01B12C92
:102E3000A12CA91688F5FB01EA0DFB1D8490912CAD
:102E4000002E02C0880C991C0A94E2F7809490949A
:102E5000FA01EA0DFB1D6490712C002E02C0660C75
:102E6000771C0A94E2F737FD05C0F60180818821BE
:102E700086298083FF2049F037303CF4F601E05882
:102E8000FF4F8081892187298083FFEFAF1ABF0A16
:102E90008FEFC81AD80ACDCF3F5F4C0F5D1F6C0F64
:102EA0007D1FA058BF4FBCCFC92ED12CFA01E60F11
:102EB000F71FA651BE4F00E810E00C191D09CC19F0
:102EC000DD09BE01660F771F41E050E06A010F2C5B
:102ED00001C0CC0C0A94EAF7592F2E2D792ECF93EE
:102EE000DF93ED01EF96EF9622968590A590FF2057
:102EF00059F08C9C4001AC9C500137302CF4E88098
:102F0000B094EB20E928E99233233AF0EC90A094B6
:102F1000EA20E828ED920C948E1711965A9529F71D
:102F20002A9551F0572D33951124E60FF11DA00F6E
:102F3000B11DC00FD11DD9CFDF91CF9111249FCEEC
:102F4000CF92EF920F93FA0104913196E4904E5F85
:102F50005F4F2223F9F0A1E0B0E03E2D377011F46D
:102F6000B0E0A0E0EE2DE695E695E695EA0FFB2FA2
:102F7000F11D0E9FD0010F9FB00D112430E0220FE4
:102F8000331FA29FF001A39FF00DB29FF00D1124FB
:102F90004E0F5F1F23E0C22E30E020E00E94B715E5
:102FA0000F91EF90CF900895CF92EF920F93CF9320
:102FB000DF93DC01FA0104913196E4904E5F5F4F9C
:102FC0002223D1F0C1E0D0E09E2D977011F4D0E023
:102FD000C0E0EE2DE695E695E695EC0FFD2FF11D90
:102FE0000E9FE0010F9FD00D11242C9FC0012D9F3B
:102FF000900D1124480F591F82E0C82E30E020E0C8
:10300000CD010E94B715DF91CF910F91EF90CF9036
:1030100008952D9A0895BC0190E080E00C94FF146F
:103020008FB18095807F669B88601C9B846008952B
:10303000480F592F511D14161506D4F580389105E7
:10304000BCF597FF02C090E080E04138510514F0D4
:1030500040E850E0481BFB0177FD379633E0F595DB
:10306000E7953A95E1F7F695FE2FEE27F795E79568
:10307000E80FF91FE651FE4F6770772781E090E077
:1030800001C0880F6A95EAF7382F213041F441508A
:1030900078F08191DF011197832B8C93F8CF809585
:1030A000415030F09191DF01119798239C93F8CF14
:1030B00008959091BB01982329F49091BC01982325
:1030C00081E009F480E0089580E00C943C1380389E
:1030D0009105B8F460347105A0F420E191E061FD40
:1030E00094E060FD990F62FD9295687F269FD00164
:1030F0001124A80FA651BE4F8C9140FF03C0892B0D
:103100008C93089590958923FBCF8F929F92AF92D5
:10311000BF92CF92DF92EF92FF920F931F93CF93C4
:10312000DF936D3089F0C090B901D090BA016A3058
:10313000D1F41092B8011092B70188E0C80ED11CEA
:10314000D092BA01C092B90181E090E0DF91CF91B5
:103150001F910F91FF90EF90DF90CF90BF90AF90B5
:103160009F908F9008950091B7011091B801E5E00C
:103170006E9FE0011124C355DE4F4801F12CF5E0AC
:10318000E12CFF1629F0CE010196FE01E490EC013E
:10319000B12CA12C4E2D4170B6016A0D7B1DC401CE
:1031A0000E946718E694FFEFAF1ABF0A88E0A816DE
:1031B000B10481F7F394EFEF8E1A9E0AF6E0FF1246
:1031C000DECF0A5F1F4F1093B8010093B701BCCF49
:1031D0000F931F93CF93DF938C01D0E0C0E0F801F1
:1031E000EC0FFD1F6491662341F08AE396E00E9494
:1031F0008518892B11F02196F2CFCE01DF91CF9166
:103200001F910F910895DF92EF92FF920F931F93FA
:10321000CF93DF937C01D22E8B01040F111DEB01A4
:1032200077FF02C0D0E0C0E0C8010134110514F0FE
:1032300080E490E0C817D9073CF44D2DBE01C701CA
:103240000E9467182196F0CFDF91CF911F910F91C7
:10325000FF90EF90DF900895CF92DF92EF92FF9270
:103260000F931F93CF93DF936B01122FEC017C011F
:10327000E40EF11CCE15DF0544F4202F412FB601DA
:10328000CE010E9403192196F5CFDF91CF911F91B6
:103290000F91FF90EF90DF90CF900895CF92DF9243
:1032A000EF92FF920F93CF93DF936C017B01C42FBA
:1032B000D22F6034710520F4202FC6010E94181807
:1032C000B7016D0F711D615071096034710528F4EB
:1032D000202F4C2FC6010E941818202F4D2FB70108
:1032E000C6010E940319C6018C0F911D202F4D2F7E
:1032F000B7010197DF91CF910F91FF90EF90DF9091
:10330000CF900C9403198091870120E0813031F037
:1033100021E0823019F0833049F422E049E651E09F
:103320006FE070E08BE190E00E94D41780918601FD
:1033300020E0813031F021E0823019F0833049F40F
:1033400022E049E651E06FE070E084E390E00E9403
:10335000D4178091850120E0813031F021E0823066
:1033600019F0833049F422E049E651E06FE070E063
:103370008DE490E00E94D4178091840120E0813098
:1033800031F021E0823019F0833049F422E049E63F
:1033900051E06FE070E086E690E00E94D4178091E3
:1033A000830120E0813031F021E0823019F0833058
:1033B00049F422E049E651E06CE270E08BE190E0F4
:1033C0000E94D4178091820120E0813031F021E009
:1033D000823019F0833049F422E049E651E06CE292
:1033E00070E084E390E00E94D4178091810120E096
:1033F000813031F021E0823019F0833049F422E04D
:1034000049E651E06CE270E08DE490E00E94D41750
:103410008091800120E0813031F021E0823019F08C
:10342000833049F422E049E651E06CE270E086E640
:1034300090E00C94D417089581E0809303018BE110
:103440008093B4018FE08093B201EDE0F1E08AE374
:1034500090E09183808380E390E093838283E3E133
:10346000F1E080E290E09183808323E030E03383D9
:103470002283E9E1F1E09183808385E090E093830A
:1034800082831092A4018AE3809306018093050150
:1034900081E1809304011092970110929E01809126
:1034A000D2018F5F8093D20110929A0183E08093C2
:1034B000270110929D0110929C011092A20110927E
:1034C00096011092950186EF9FEF909302018093F1
:1034D0000101109299011092A6011092A50180ECB1
:1034E0009FEF9093200180931F0180E49FEF9093C2
:1034F00024018093230180E89FEF90932201809321
:1035000021018BEF9FEF90930801809307011092A8
:10351000AB01089520919501233009F072C081E03C
:10352000809303019DE19093B4019FE09093B201D9
:103530004AE350E050930E0140930D0140E350E008
:103540005093100140930F0140E250E0509314015A
:103550004093130163E070E07093160160931501CE
:1035600050931A014093190145E050E050931C011B
:1035700040931B011092A4019AE39093060190934B
:10358000050191E1909304011092970110929E0120
:103590009091D2019F5F9093D20110929A01209353
:1035A00027011092A201109296011092950126EF28
:1035B0003FEF309302012093010110929901109284
:1035C000A6011092A50120EC3FEF3093200120933B
:1035D0001F0120E43FEF309324012093230120E8D2
:1035E0003FEF30932201209321018093D3018093F8
:1035F000D1018BEF9FEF9093080180930701109208
:10360000AB010895089590E080E008958F929F9215
:10361000AF92BF920F931F93CF93DF93CDB7DEB7D7
:10362000A1970FB6F894DEBF0FBECDBF19A24230EE
:1036300008F44AE08E010F5D1F4F842E912CB12CAF
:10364000A12CA50194010E945937E62FB901CA01A6
:10365000EA3044F5E05DD801EE938D01232B242B55
:10366000252B79F790E080E0109769F0FD0101903B
:103670000020E9F73197AF014A1B5B0BBD018AE3DC
:1036800096E00E94AD14A1960FB6F894DEBF0FBE6F
:10369000CDBFDF91CF911F910F91BF90AF909F90C1
:1036A0008F900895E95CD7CFCF92DF92EF92FF928F
:1036B000CF93DF936C01990FEE08FF08F7FE19C056
:1036C0006DE28AE396E00E948518EC016627772771
:1036D000CB016C197D098E099F094AE00E94061BE7
:1036E0008C0F9D1FDF91CF91FF90EF90DF90CF90D7
:1036F00008954AE0C701B601DF91CF91FF90EF90A6
:10370000DF90CF900C94061BCF930E948319809179
:10371000B001C091B401813009F079C06091B2016B
:103720006350770B20E049E651E0EC2FE250FF0BAD
:10373000CF010E94D41780E40E945918882329F0F1
:10374000C73618F4C75EC093B40180E20E945918CE
:10375000882339F08091B4018F3118F0895180931A
:10376000B40180E10E945918882339F08091B20198
:103770008F3019F48CE28093B20180E80E945918CE
:10378000882339F08091B2018C3219F48FE0809354
:10379000B2018091B4018D3109F04EC08091B20127
:1037A0008F3009F08AC08CE690E09093B801809346
:1037B000B7011092BA011092B90180919C019091C9
:1037C0009D010E94541B83E590E09093B801809383
:1037D000B7011092BA011092B9018091CE01909177
:1037E000CF010E94541B84E00E945918882321F1C4
:1037F00080919C0190919D019093CF018093CE0187
:103800008091B0018130A1F48093870115C082308E
:1038100031F46091B2016350770B21E084CF8330A3
:1038200009F089CF6091B2016350770B22E07BCF22
:10383000823051F3833041F38091B4018633E9F54E
:103840008091B2018F3009F079C08CE690E09093BE
:10385000B8018093B7011092BA011092B90180911A
:103860009C0190919D010E94541B83E590E09093F0
:10387000B8018093B7011092BA011092B9018091FA
:10388000CC019091CD010E94541B84E00E945918F4
:10389000882399F080919C0190919D019093CD0196
:1038A0008093CC018091B001813019F4809386011E
:1038B00004C08230D9F38330C9F38091B4018F34CE
:1038C000E9F58091B2018F3009F079C08CE690E083
:1038D0009093B8018093B7011092BA011092B90188
:1038E00080919C0190919D010E94541B83E590E082
:1038F0009093B8018093B7011092BA011092B90168
:103900008091CA019091CB010E94541B84E00E94D7
:103910005918882399F080919C0190919D01909372
:10392000CB018093CA018091B001813019F480935A
:10393000850104C08230D9F38330C9F38091B4018A
:103940008836E9F58091B2018F3009F079C08CE6B4
:1039500090E09093B8018093B7011092BA01109251
:10396000B90180919C0190919D010E94541B83E5B7
:1039700090E09093B8018093B7011092BA01109231
:10398000B9018091C8019091C9010E94541B84E043
:103990000E945918882399F080919C0190919D0173
:1039A0009093C9018093C8018091B001813019F4CE
:1039B0008093840104C08230D9F38330C9F38091AD
:1039C000B4018D31E9F58091B2018C3209F079C0F2
:1039D0008CE690E09093B8018093B7011092BA0101
:1039E0001092B90180919C0190919D010E94541BFD
:1039F00083E590E09093B8018093B7011092BA01EB
:103A00001092B9018091C6019091C7010E94541B88
:103A100084E00E945918882399F080919C0190912C
:103A20009D019093C7018093C6018091B0018130C0
:103A300019F48093830104C08230D9F38330C9F331
:103A40008091B4018633E9F58091B2018C3209F09E
:103A500079C08CE690E09093B8018093B701109202
:103A6000BA011092B90180919C0190919D010E9430
:103A7000541B83E590E09093B8018093B7011092B6
:103A8000BA011092B9018091C4019091C5010E94C0
:103A9000541B84E00E945918882399F080919C015E
:103AA00090919D019093C5018093C4018091B001D4
:103AB000813019F48093820104C08230D9F38330BD
:103AC000C9F38091B4018F34E9F58091B2018C3251
:103AD00009F078C08CE690E09093B8018093B7012C
:103AE0001092BA011092B90180919C0190919D01B0
:103AF0000E94541B83E590E09093B8018093B70136
:103B00001092BA011092B9018091C2019091C30143
:103B10000E94541B84E00E945918882399F08091D8
:103B20009C0190919D019093C3018093C20180916B
:103B3000B001813019F48093810104C08230D9F33F
:103B40008330C9F38091B4018836E1F58091B201E8
:103B50008C32C1F58CE690E09093B8018093B70168
:103B60001092BA011092B90180919C0190919D012F
:103B70000E94541B83E590E09093B8018093B701B5
:103B80001092BA011092B9018091C0019091C101C7
:103B90000E94541B84E00E9459188823F1F0809100
:103BA0009C0190919D019093C1018093C0018091EF
:103BB000B001813019F48093800104C08230D9F3C0
:103BC0008330C9F384E00E945918882331F01092A1
:103BD000D10110929D0110929C01CF910895682F00
:103BE00070E090E080E04AE00C94061B0C941137E2
:103BF0002F923F925F926F927F928F929F92AF929D
:103C0000BF92CF92DF92EF92FF920F931F93CF93C9
:103C1000DF9381EC80937C0085B1806F85B984B19E
:103C2000877E84B984B1876E84B95E9A5F988AB1C1
:103C3000806D8AB9769A6E9881B3806F81BB8998BE
:103C400080B38D7080BB80E58CBD81E08DBD85E04B
:103C500090E00E940B185F9A85E090E00E940B189C
:103C60005E985C98ECE5F1E084918EBD00000DB4A7
:103C700007FEFDCF319641E0E936F407A9F75C9ADB
:103C800081E8809364008091650081608093650085
:103C90000E9464180E94101887FF15C05C9885EA7E
:103CA0008EBD00000DB407FEFDCF5C9A2E982F98B4
:103CB0002D988091640080628093640081E083BFCE
:103CC000889513BEFCCF0E94101882FF48C02D9823
:103CD0000E94101884788438E1F40E94091888EC56
:103CE00090E00E940B182F9882E090E00E9411371C
:103CF0008F3F29F06FEF82E090E00E94193784EF48
:103D000091E00E940B182F9A0E9410188478843832
:103D1000D9F30E94101884718431E1F40E940918CB
:103D200088EC90E00E940B182E9882E090E00E94B0
:103D30001137882329F060E082E090E00E94193773
:103D400084EF91E00E940B182E9A0E941018847143
:103D50008431D9F388EC90E00E940B18B4CF0E9414
:103D6000091882E090E00E94F61D8823D9F13E9A5E
:103D70003F9A81E090E00E94F61D81FF11C0582F0C
:103D80005470552E82FD2E98C1EFDFEF08E010E051
:103D90000E94101886FF29C02E9A2F9A0E94091897
:103DA00082E390E00E940B180E9410188111F8CF56
:103DB00080E180930001109290008AE0809391004E
:103DC000DF91CF911F910F91FF90EF90DF90CF90F7
:103DD000BF90AF909F908F907F906F905F903F903B
:103DE0002F9008953E983F98C4CF552029F0C430B5
:103DF000D10511F42E9A2F9881E00E943C139E0168
:103E0000D7FF04C0222733272C1B3D0B27703327F5
:103E1000CE01D7FD079653E0959587955A95E1F722
:103E2000D7FF05C00197F801E21BF30B9F01BC010E
:103E30007695762F66277795679566517E4FB0E029
:103E4000A0E03801621A730A8E3FFFEF9F0709F462
:103E50003BC07B0150E040E0FD01E455FF4F5F01B6
:103E60004B01F0E88F0E911C8F3F980779F0F50118
:103E7000E40FF51FE491F0E06F01022E01C0CC0CBD
:103E80000A94EAF7F701D488CD28C48A21153105B0
:103E900099F0F501E40FF51FE4916401C40ED51EFD
:103EA000F0E01F01062C02C0359427940A94E2F733
:103EB000F60134882328248A4F5F5F4FFFEFEF1A03
:103EC000FF0A4835510581F60196A85ABF4F605840
:103ED0007F4FA03BB10509F0B7CF0E9464188FE077
:103EE00090E00E940B182196C931D10509F050CFFE
:103EF000552011F02F9A2D9880E991E00E940B181F
:103F00000E94091881E090E00E94F61D80FF48CFD2
:103F10008AE090E00E94F61D9FEF980F9E3F08F008
:103F20003FCF22E330E03093B8012093B70128E37C
:103F300030E03093BA012093B901CBE0D0E0682F94
:103F40008AE396E00E948518CE010E94F61D219614
:103F5000C131D105A1F70E94641888EE93E00E9458
:103F60000B181ECF1F920F920FB60F9211248F9332
:103F70009F938091E1009091E100937F9093E10005
:103F800083FF0FC01092E90091E09093EB00109234
:103F9000EC0092E39093ED001092E90198E0909389
:103FA000F00082FF22C093E09093E9009091F2002C
:103FB000992319F09AE39093E8009091DA019923FC
:103FC00041F09091DA0191509093DA01911101C082
:103FD0005D9A9091E801992341F09091E801915008
:103FE0009093E801911101C0289A84FF18C0809134
:103FF000E2008E7E81608093E2008091E1008F7EFE
:104000008093E1008091DB018E7E80618093DB01F3
:104010009F918F910F900FBE0F901F90189580FF6A
:10402000F7CF8091E2008E7E80618093E2008091E4
:10403000E1008E7E8093E1008091DB018E7E8160C5
:10404000E5CF1F920F920FB60F921124CF92DF92FD
:10405000EF92FF920F931F932F933F934F935F9392
:104060006F937F938F939F93AF93BF93EF93FF9340
:10407000CF93DF93CDB7DEB76C97DEBFCDBF109285
:10408000E9008091E80083FF25C068E0CE014596F5
:104090000E94A01482EF8093E8008D8987FF39C0C9
:1040A0009091E80090FFFCCF982F907609F034C1F2
:1040B0009E894F89588D2F89F88C911131C0803895
:1040C00061F58091D9018093F1001092F1008EEF9B
:1040D0008093E8006C960FB6F894DEBF0FBECDBF9C
:1040E000DF91CF91FF91EF91BF91AF919F918F9110
:1040F0007F916F915F914F913F912F911F910F9100
:10410000FF90EF90DF90CF900F900FBE0F901F9019
:1041100018959EEF9093E800C7CF1092F100D5CF8D
:10412000913059F48111D3CF4130510581F68091FE
:10413000D9018D7F8093D901CACF933049F4811181
:10414000C6CF4130510519F68091D9018260F2CF76
:10415000953041F48091E80080FFFCCF20682093E7
:10416000E300B5CF963009F0A9C00B8D1C8D22E07D
:104170001092E9001092D7011092D601F2122EC0CF
:104180001092D5011092D4010E946F141F8299E001
:104190009983FA8291E09E8390EA98879AEF9987B3
:1041A0002091D6013091D701275F3F4F3C832B836D
:1041B0008D831092E9001092D7011092D6011093CE
:1041C000D5010093D40149E050E0BE016F5F7F4FFD
:1041D00080E00E9449140E946F1479CF1093D5019A
:1041E0000093D4010E948613DC0112960D911C915C
:1041F0000115110509F451C1D801ED91FC9104801C
:10420000F581E02DBE016B5E7F4FC80109950097D7
:1042100009F03EC1F80100851185EACFF3E0FF12F5
:104220000EC08F89882309F440C0823061F440E8D1
:1042300060E181E196E20E949D22811148CF81E2F6
:104240008093EB0047CF813029F440E86BE085E0B4
:1042500096E2F1CF833099F70E948613DC01129623
:10426000ED90FC908E010F5F1F4F6801E114F10487
:1042700079F0D701ED91FC910680F781E02DB8012E
:10428000C7010995080F111DF701E084F184EECFF5
:10429000D8011C92F60101900020E9F73197BF0187
:1042A0006C197D0940E0C601C6CF6FEE75E2FB01D7
:1042B000449150E080E80E94491409CF973009F4F6
:1042C000BECF983021F481E08093F10000CF993087
:1042D00009F0FDCE837009F0B2CFE6E5F1E081E0B0
:1042E00031E096E32191222371F08093E90030932D
:1042F000EB00DF0111972C912093EC009093ED00DF
:104300008F5F873079F78EE78093EA001092EA009A
:104310008F898093E901DBCE8B8D9C8D1092E90013
:104320001092D7011092D6019093D5018093D401B9
:10433000898D811192C08E899D89913A49F481328B
:1043400009F07DCF47E050E06EE271E080E0B3CF4E
:10435000913209F074CF833269F48F89988DB0E07F
:10436000A0E080932A0190932B01A0932C01B0939D
:104370002D01ADCE803269F48091E80082FFFCCF40
:1043800067E08EE291E00E94A0148BEF8093E8003A
:104390009ECE823209F09BCE8F8980933501EEEF5D
:1043A000FFE7859194918B3F9C4D51F1E0E0F8E05F
:1043B00080912E0190912F01A0913001B091310197
:1043C000803B9440A105B105F1F48091350180FD59
:1043D0001AC0EE3F8AE0F80789F587E797E79183EF
:1043E0008083809160008093D80188E19BE00FB6C4
:1043F000F894A895809360000FBE9093600067CEFC
:10440000EEEFFAE0D5CF808191818737974709F0A9
:104410005ECEA89580916000886180936000809155
:10442000D80180936000EE3F2AE0F20789F0809186
:10443000FE0A9091FF0A9183808349CE8081918109
:104440008737980751F29093FF0A8093FE0AC5CFF1
:104450001092FF0A1092FE0A3ACE0E948613DC01E7
:1044600012960D911C910115110509F4E8CED801A1
:10447000ED91FC910190F081E02DBE016B5E7F4FCC
:10448000C8010995811123CEF80100851185EBCF74
:10449000181619060CF41BCED2CEF1E0FF12BECED8
:1044A00063EF75E204CF1F920F920FB60F921124A3
:1044B0002F933F938F939F93AF93BF9380918D01E1
:1044C00090918E01A0918F01B0919001309188015F
:1044D00023E0230F2D3758F50196A11DB11D209320
:1044E000880180938D0190938E01A0938F01B093EA
:1044F00090018091890190918A01A0918B01B091E6
:104500008C010196A11DB11D8093890190938A01B0
:10451000A0938B01B0938C01BF91AF919F918F912C
:104520003F912F910F900FBE0F901F90189526E886
:10453000230F0296A11DB11DD2CFEF92FF920F93D0
:104540001F93CF93DF93F82E192FE62E042F81E0CF
:10455000860F880F0E941B1483E00E941B14CF2D2E
:10456000D12FEC0EFD2EF11CCE15DF05B9F007FFA3
:1045700013C0FE0184910E941B14182F80E00E943A
:104580001B14812321968111EFCFDF91CF911F91D1
:104590000F91FF90EF9008958881EDCF81E0F5CFE6
:1045A000EAEEF5E01382128288EE93E0A0E0B0E03C
:1045B00084839583A683B78380E691E0918380838B
:1045C0008FEF9FEF95878487EAE3F6E013821282EC
:1045D00082E791E0918380830895CF93DF93CDB7F5
:1045E000DEB7EF970FB6F894DEBF0FBECDBF78945D
:1045F00084B5826084BD84B5816084BD85B58260E8
:1046000085BD85B5816085BD80916E008160809398
:104610006E00109281008091810082608093810001
:104620008091810081608093810080918000816011
:1046300080938000809191008260809391008091AE
:1046400091008160809391008091900081608093BF
:1046500090008091C10084608093C1008091C1006E
:1046600082608093C1008091C10081608093C1000D
:104670008091C30081608093C3008091C0008260FC
:104680008093C0008091C20081608093C2008091BD
:104690007A00846080937A0080917A0082608093AF
:1046A0007A0080917A00816080937A0080917A000C
:1046B000806880937A001092E9011092D9011092DB
:1046C000DB018091D70081608093D70080EA8093DE
:1046D000D80089B5806189BD89B5826089BD09B47A
:1046E00000FEFDCF61E070E080E090E00E94FF14EA
:1046F0008091D8008F7C80618093D8008091E00009
:10470000807F8093E0008091E1008E7E8093E100C5
:104710008DE08093E200559A209A0E94F81D73E084
:10472000872E912C8FB7F89440918D0150918E0176
:1047300060918F01709190018FBF809191018823CA
:1047400049F01092910180E090E0892B59F30E948A
:104750000000E5CF80919201F42EF81A8F2D9091F0
:104760000001F91640F48F5F891768F781E083BF75
:10477000889513BEE8CF81E0809391014093920128
:104780008091AC019091AD0101969093AD01809321
:10479000AC018091BD01882339F081508093BD0127
:1047A000811102C0109290008091BC018093BB01E6
:1047B0000E9410188093BC0180E0EAEEF1E08111C4
:1047C0008FEF002481938193819381930394D1F798
:1047D0001092BA011092B9011092B8011092B7016B
:1047E0001091D301123011F40C94B92C48F4112318
:1047F00009F48AC0113009F4F9C00E946418A3CFEB
:10480000143011F40C94B43510F40C949B3515301D
:10481000A1F780E290E09093B8018093B7018FE018
:1048200090E09093BA018093B9018AE59DE10E94DE
:10483000E8188DE290E09093B8018093B7018EE183
:1048400090E09093BA018093B90183E59DE10E94C5
:10485000E8188AE590E09093B8018093B70187E368
:1048600090E09093BA018093B9018CE49DE10E949D
:10487000E818809128018130E1F580910101909143
:104880000201019690930201809301018B3F9F4F9B
:104890005CF41093BD0180E48093900083EC99E078
:1048A000909399008093980080910101909102016A
:1048B0008D3F9F4F60F085E08093BD0180E4809341
:1048C000900084E09DE090939900809398008091FF
:1048D0000101909102010A9760F488E08093BD0184
:1048E00080E4809390008FE097E29093990080930A
:1048F000980084E00E945918882309F47ECF0E9412
:104900001C1A81E00C94113520E04BEA51E270E072
:1049100060E090E080E00E94D41780E10E94591886
:10492000882339F080912901823018F48F5F8093B9
:10493000290180E80E945918882339F080912901C3
:10494000823018F081508093290110912901113093
:10495000F1F420E044EA51E26FE170E08AE390E094
:104960000E94D41784E00E94591881111093D3013A
:1049700080912801813009F040CF01E022E042E03F
:104980006BE270E087E690E00E942C1936CF12307F
:1049900079F71091280120E044EA51E269E270E0E1
:1049A00081E690E00E94D41784E00E945918882381
:1049B00021F0123011F41092280184E00E9459185D
:1049C000882339F080912801813019F482E08093A6
:1049D000280184E00E945918882351F2809128010F
:1049E0008111C6CF81E080932801C2CF20E042EA46
:1049F0005DE170E060E090E080E00E94D41780917B
:104A0000D2018D3051F48091D101811106C084E032
:104A10000E94591881111093D0012091BE0130914C
:104A2000BF01253F41E034073CF08091B601811180
:104A300028C583E08093B5018091B501853009F0E8
:104A4000FFC380912801813009F072C18091AF01CC
:104A50009091D101911102C0882319F0823009F0A0
:104A600067C18091AC019091AD01B4010E948A3779
:104A7000892B29F48091AE018F5F8093AE018091E4
:104A8000AE018A3060F488E08093BD0180E48093B9
:104A900090008BE09EE19093990080939800809124
:104AA000AE018051843060F485E08093BD0180E4E4
:104AB000809390008DEE93E19093990080939800FD
:104AC0008091AE018A51843060F485E08093BD010D
:104AD00080E4809390008DEE93E190939900809311
:104AE00098008091AE018452843060F485E0809318
:104AF000BD0180E4809390008DEE93E19093990046
:104B0000809398008091AE018952893060F488E0EA
:104B10008093BD0180E4809390008BE09EE19093B0
:104B20009900809398008091AE018853843060F49E
:104B300085E08093BD0180E4809390008DEE93E149
:104B400090939900809398008091AE0182548430B4
:104B500060F485E08093BD0180E4809390008DEE49
:104B600093E190939900809398008091AE018C54CA
:104B7000853060F485E08093BD0180E480939000EF
:104B80008BED97E290939900809398008091AE010D
:104B900081558A3060F488E08093BD0180E4809381
:104BA00090008BE09EE19093990080939800809113
:104BB000AE018056843060F485E08093BD0180E4CE
:104BC000809390008DEE93E19093990080939800EC
:104BD0008091AE018A56843060F485E08093BD01F7
:104BE00080E4809390008DEE93E190939900809300
:104BF00098008091AE018457843060F485E0809302
:104C0000BD0180E4809390008DEE93E19093990034
:104C1000809398008091AE018957843060F483E0DE
:104C20008093BD0180E4809390008BE09EE190939F
:104C30009900809398008091AE018E57843060F483
:104C400083E08093BD0180E4809390008BE09EE13F
:104C500090939900809398008091AE01835884309E
:104C600060F483E08093BD0180E48093900080EC49
:104C70009AE190939900809398008091AE018858B2
:104C8000843060F483E08093BD0180E480939000E1
:104C900081ED97E190939900809398008091AE0107
:104CA0008D58843060F483E08093BD0180E480936C
:104CB000900082E796E1909399008093980080910C
:104CC000AE018259843060F483E08093BD0180E4BA
:104CD0008093900081ED97E19093990080939800E4
:104CE0008091AE018759843060F483E08093BD01E8
:104CF00080E48093900080EC9AE1909399008093F7
:104D000098008091AE018C59843060F483E08093E8
:104D1000BD0180E4809390008BE09EE19093990028
:104D2000809398008091AE01873D11F41092AE01FE
:104D300020E04AEE5CE16BE070E082E090E00E94EF
:104D4000D4170091BE011091BF01053F61E0160725
:104D5000ACF021E04AEE5CE16CE170E082E090E0D2
:104D60000E94D417013B14404CF022E04AEE5CE173
:104D70006DE270E082E090E00E94D4178091D10152
:104D80008111DAC10E94831980E20E945918882398
:104D900049F08091B4018C3129F481E0809326019F
:104DA0001092B3018091B301813009F013C1F090EA
:104DB000B2011091B4016F2D70E000E029E049E0EC
:104DC000812F90E00E944E1920E046EB5CE167E302
:104DD00070E086E190E00E94D41780E40E945918A8
:104DE000882329F0173618F4175E1093B40180E277
:104DF0000E945918882339F08091B4018F3118F03E
:104E000089518093B40180E10E945918882331F0C0
:104E100080E1F81203C08EE28093B20180E80E9424
:104E20005918882339F08091B2018E3219F480E14B
:104E30008093B2018091B4018C31B1F48091B201C0
:104E4000803191F48EE190E09093B8018093B701A6
:104E500088E390E09093BA018093B9018091CE01EC
:104E60009091CF010E94541B8091B4018533B1F41D
:104E70008091B201803191F48EE190E09093B8017D
:104E80008093B70188E390E09093BA018093B901D1
:104E90008091CC019091CD010E94541B8091B4016E
:104EA0008E34B1F48091B201803191F48EE190E0C2
:104EB0009093B8018093B70188E390E09093BA0192
:104EC0008093B9018091CA019091CB010E94541B3B
:104ED0008091B4018736B1F48091B201803191F4B0
:104EE0008EE190E09093B8018093B70188E390E061
:104EF0009093BA018093B9018091C8019091C90142
:104F00000E94541B8091B4018C31B1F48091B201A4
:104F10008E3291F48EE190E09093B8018093B701C6
:104F200088E390E09093BA018093B9018091C60123
:104F30009091C7010E94541B8091B4018533B1F454
:104F40008091B2018E3291F48EE190E09093B8019D
:104F50008093B70188E390E09093BA018093B90100
:104F60008091C4019091C5010E94541B8091B401AD
:104F70008E34B1F48091B2018E3291F48EE190E0E2
:104F80009093B8018093B70188E390E09093BA01C1
:104F90008093B9018091C2019091C3010E94541B7A
:104FA0008091B4018736B1F48091B2018E3291F4D0
:104FB0008EE190E09093B8018093B70188E390E090
:104FC0009093BA018093B9018091C0019091C10181
:104FD0000E94541B80E40E945918882371F080912C
:104FE0002601813051F4109226018093B3018CE1A7
:104FF0008093B40180E18093B201F090260191E0AA
:10500000F9129AC020E04CE85CE167E370E086E1C9
:1050100090E00E94D4171091B101111133C000E04B
:105020002EE04EE06CE070E083E090E00E944E19CC
:105030008EE190E09093B8018093B70188E390E00F
:105040009093BA018093B90189E89CE10E94E81825
:1050500088E290E09093B8018093B7018AE090E0F5
:105060009093BA018093B9018EE79CE10E94E81801
:1050700084E00E945918882329F0F092B00182E060
:105080008093D301E090BE01F090BF01A5EFEA1636
:10509000A1E0FA06B4F1113009F0FCC100E02EE005
:1050A0004EE06DE170E083E090E00E944E198EE1E9
:1050B00090E09093B8018093B70188E390E09093DB
:1050C000BA018093B9018BE79CE10E94E81888E25D
:1050D00090E09093B8018093B7018AE090E09093BC
:1050E000BA018093B9018FE69CE10E94E81884E040
:1050F0000E945918882329F082E08093B0018093A0
:10510000D30180E80E945918882329F0112319F04F
:1051100011501093B10180E10E945918882361F069
:105120008091B101823040F425EFE21621E0F206D1
:105130001CF08F5F8093B1018091D101813009F023
:105140007FC08091AF01823011F40E94841B809156
:10515000AF01813009F041C000E028E24EE66BE08B
:1051600070E08AE090E00E942C198FE090E090932C
:10517000B8018093B7018CE090E09093BA018093DE
:10518000B9018FE49CE10E94E81881E190E09093DE
:10519000B8018093B70189E190E09093BA018093C0
:1051A000B9018EE39CE10E94E81880E290E09093C0
:1051B000B8018093B70185E290E09093BA018093A3
:1051C000B90184E39CE10E94E81884E00E94591828
:1051D0008823B1F182E08093AF018091AF0181110A
:1051E0002FC000E02BE14EE66BE070E08AE090E03B
:1051F0000E942C1909E110E01093B8010093B70147
:105200008CE090E09093BA018093B90185E29CE133
:105210000E94E81888E290E09093B8018093B7016B
:105220001093BA010093B9018BE19CE10E94E81848
:1052300084E00E945918882319F081E08093AF011F
:105240008091D2018D3009F09EC08091D1018111F1
:105250009AC083E08093AF018091AC019091AD0141
:10526000B4010E948A37892B29F48091AB018F5FAA
:105270008093AB0180912801813009F043C0809177
:10528000AB018A3060F488E08093BD0180E48093B4
:10529000900086EF9EE09093990080939800809113
:1052A000AB018051893060F488E08093BD0180E4D7
:1052B000809390008FED9BE09093990080939800ED
:1052C0008091AB018452823060F483E08093BD0111
:1052D00080E48093900086EF99E09093990080930A
:1052E00098008091AB0187528B3060F488E0809306
:1052F000BD0180E48093900080EE98E09093990047
:1053000080939800109226011092B30100E02FE2E2
:105310004DE66BE070E08AE090E00E942C198091ED
:10532000D0018111F5C081E190E09093B8018093A4
:10533000B7018DE090E09093BA018093B9018AE0C3
:105340009CE10E94E8188DE190E09093B801809371
:10535000B7018EE190E09093BA018093B9018DEF8F
:105360009BE10E94E81885E290E09093B801809359
:10537000B70188E290E09093BA018093B90182EF7F
:105380009BE10E94E8188091B501823009F45EC269
:1053900008F098C1882309F4DBC1813009F407C201
:1053A00082E090E09093B8018093B7011092BA0127
:1053B0001092B9018091D2010E94EF1D8DE090E022
:1053C0009093B8018093B7011092BA011092B9017D
:1053D00041E050E06AE771E08AE396E00E94AD1494
:1053E00084E190E09093B8018093B7011092BA01E4
:1053F0001092B90142E050E06CE771E08AE396E078
:105400000E94AD148091CE019091CF012091CC01EA
:105410003091CD01820F931F2091CA013091CB01B1
:10542000820F931F2091C8013091C901820F931FF1
:105430002091C6013091C701820F931F2091C401B2
:105440003091C501820F931F2091C2013091C30199
:10545000820F931F2091C0013091C101820F931FD1
:105460009093BF018093BE012BE230E03093B801EE
:105470002093B7011092BA011092B9010E94541BF7
:10548000BCC9213B34400CF4D7CA813009F0D4CADE
:1054900084E0D0CAE1EBEE16E4E0FE060CF431CE77
:1054A000123009F02ECE00E02EE04EE06EE270E009
:1054B00083E090E00E944E198EE190E09093B80155
:1054C0008093B70188E390E09093BA018093B9018B
:1054D0008CE69CE10E94E81888E290E09093B80185
:1054E0008093B7018AE090E09093BA018093B9016C
:1054F00081E69CE10E94E81884E00E945918882304
:1055000009F4FFCD83E08093B0011093D301F9CD6E
:10551000813009F038CF01E024E144E165E170E039
:1055200084E190E00E944E1924E144E165E170E0DD
:105530008BE290E00E944E1924E144E165E170E0C5
:1055400082E490E00E944E1924E144E165E170E0BC
:1055500089E590E00E944E1980E40E945918882342
:1055600039F080912501893518F4895E80932501F1
:1055700080E20E945918882339F0809125018631F4
:1055800018F08751809325018EE190E09093B80147
:105590008093B7018CE090E09093BA018093B901B9
:1055A00085EE9BE10E94E818109125018091A901E8
:1055B0009091AA018A3F9105DCF023E043EF5AE184
:1055C00065E170E084E190E00E94D417153181F428
:1055D00087E290E09093B8018093B7018DE290E06C
:1055E0009093BA018093B90189EE9AE10E94E8187C
:1055F0008091A8018931D8F022E043EF5AE165E1BA
:1056000070E08BE290E00E94D4171C3281F484E1B8
:1056100090E09093B8018093B7018DE290E0909371
:10562000BA018093B90189ED9AE10E94E81880914E
:10563000A70181111BC020E043EF5AE165E170E052
:1056400082E490E00E94D417133481F481E390E067
:105650009093B8018093B7018DE290E09093BA01E6
:105660008093B90182ED9AE10E94E8188091BE0111
:105670009091BF01813D9740DCF021E043EF5AE17A
:1056800065E170E089E590E00E94D4171A3581F455
:1056900088E290E09093B8018093B7018DE290E0AA
:1056A0009093BA018093B90188EC9AE10E94E818BE
:1056B00001E022E142E166E170E0812F90E00E948A
:1056C0004E1961CE833009F410C1843009F068CEE0
:1056D00000E024E246E66BE070E08FE090E00E949C
:1056E0002C1905E110E01093B8010093B7018FE089
:1056F00090E09093BA018093B90183EF99E10E9401
:10570000E8181093B8010093B70189E190E09093F5
:10571000BA018093B90183EE99E10E94E81883E20F
:1057200090E09093B8018093B7019093BA01809371
:10573000B90187ED99E10E94E81884E00E945918A8
:10574000882309F42DCE85E08093B50182E00EC157
:1057500000E02DE244E66BE070E08FE090E00E9414
:105760002C1903E210E01093B8010093B70182E115
:1057700090E09093BA018093B9018DEB9AE10E9479
:10578000E8181093B8010093B7011093BA01009381
:10579000B90182EB9AE10E94E81884E00E9459184E
:1057A000882309F4FDCD81E08093B501F9CD00E0B7
:1057B0002FE24EE66BE070E08AE090E00E942C1948
:1057C00000E110E01093B8010093B7018FE090E082
:1057D0009093BA018093B90181EA9AE10E94E81896
:1057E0008EE090E09093B8018093B70189E190E05A
:1057F0009093BA018093B9018FE89AE10E94E8186A
:1058000087E190E09093B8018093B70183E290E044
:105810009093BA018093B90180E89AE10E94E81858
:105820001093B8010093B7018DE290E09093BA0114
:105830008093B9018FE69AE10E94E81884E00E9403
:105840005918882309F4ACCD82E0AECF00E02FE2F6
:105850004EE66BE070E08AE090E00E942C190EE0CA
:1058600010E01093B8010093B7018FE090E090939F
:10587000BA018093B9018DE59AE10E94E81810936E
:10588000B8010093B70189E190E09093BA01809349
:10589000B9018BE49AE10E94E81887E190E09093C7
:1058A000B8018093B70183E290E09093BA018093AE
:1058B000B9018CE39AE10E94E8188DE190E09093A1
:1058C000B8018093B7018DE290E09093BA01809384
:1058D000B90180E39AE10E94E81884E00E94591817
:1058E000882309F45DCD85E05FCF00E024E246E641
:1058F0006BE070E08FE090E00E942C1905E110E071
:105900001093B8010093B7018FE090E09093BA0133
:105910008093B90180E29AE10E94E8181093B801DF
:105920000093B70189E190E09093BA018093B901A7
:1059300080E19AE10E94E8188EE190E09093B8012E
:105940008093B70183E290E09093BA018093B9010C
:1059500083E09AE10E94E81884E00E9459188823A5
:1059600009F41ECD85E08093B50181E08093B601F6
:1059700017CDE0902301F090240120E045ED51E1A6
:10598000B70190E080E00E94D417C0902101D09030
:10599000220121E045ED51E1B60190E080E00E9456
:1059A000D41740911F015091200159AF48AF20E01A
:1059B00043ED59E068AD79AD8091A5019091A601C4
:1059C0000E94D41720E045E659E06CE270E090E0D8
:1059D00080E00E94A01720E046EB5CE167E370E006
:1059E00087E690E00E94D41701E02EE048E062E3F1
:1059F00070E082E190E00E942C1950E4C516D104B9
:105A000031F480EC9FEF909322018093210160E4B8
:105A1000E616F10431F480EC9FEF9093240180931B
:105A200023018091A401E82FF0E0E65CFE4F908115
:105A3000A92EB12CB0921C01A0921B012091AC01A7
:105A40003091AD01A901417055275BAF4AAF20FDF0
:105A500032C04091190150911A014835510554F452
:105A60009091A301911106C04F5F5F4F50931A01AF
:105A7000409319014091190150911A01483551057F
:105A800071F491E09093A3019091A301913051F4AE
:105A90004150510950931A014093190103C04132FA
:105AA000510594F74091190150911A014032510566
:105AB00011F41092A3010091190110911A012370A1
:105AC0003327232B71F40C3311050CF0B8C19091DE
:105AD000A30191110C9457368A3118F48F5F80938B
:105AE000A40184E00E945918882339F08091A20112
:105AF000811103C081E08093A201809115019091F2
:105B000016018034910511F41092A201F090A101C8
:105B1000FFAA20910F01309110012F33310591F42C
:105B2000FF2031F020E330E03093100120930F018B
:105B3000209113013091140130930E0120930D0137
:105B40001092A2017091A201713009F085C18034D8
:105B500091052CF40196909316018093150186E02F
:105B6000EDE0F1E0DE019B9601900D928A95E1F760
:105B700080910D0190910E0160900F0170901001C5
:105B8000409111016091120126E0E3E1F1E0DE01B4
:105B9000959601900D922A95E1F7E0911301F0910D
:105BA0001401F0901701FBAAF0901801FCAA480F0D
:105BB000592F511DE417F507CCF59F01FBA82F0DB8
:105BC000311D8217930794F520911501309116012C
:105BD000D301A60FB11D2A173B0744F5D901FCA834
:105BE000AF0DB11D6A167B060CF57130F9F4DC01BE
:105BF0001197EA17FB072CF4DF011196A817B907D4
:105C00004CF0DC011196AE17BF0724F090931401FD
:105C1000809313012150310930931601209315010F
:105C200022E02093A20121E02093A00126E0EDE0F4
:105C3000F1E0DE015F9601900D922A95E1F726E0F2
:105C4000E3E1F1E0DE01599601900D922A95E1F72A
:105C5000209113013091140120901501309016010C
:105C600024173507E4F4F901FBA8EF0DF11D8E1799
:105C70009F07ACF4F301E60FF11D2E163F067CF4EE
:105C8000F101FCA8EF0DF11D6E167F0644F4F10141
:105C90003E96E615F7051CF02817390774F0F10158
:105CA0007096E615F705A1F4F9013896E817F9079B
:105CB0007CF43696E817F9075CF01092A0012750A3
:105CC0003109309314012093130121E02093A201A4
:105CD00026E0EDE0F1E0DE01539601900D922A9569
:105CE000E1F726E0E3E1F1E0DE011D9601900D927F
:105CF0002A95E1F7209113013091140124173507FB
:105D0000ECF4A901FBA84F0D511D84179507B4F4BD
:105D1000660D772D711D2616370684F4A101FCA8A7
:105D20004F0D511D641675064CF4A101425F5F4F83
:105D3000461557051CF08217930784F0A101405FB8
:105D40005F4F46155705A9F4AC01485F5F4F4217F6
:105D500053077CF40E96821793075CF01092A00113
:105D6000295F3F4F309314012093130181E080930A
:105D7000A201C80107969501215F3F4F3DAF2CAFAF
:105D800060E4462E512C481A590A57FE03C051941C
:105D9000419451084CAD5DAD441655060CF46BC0F2
:105DA000813491050CF06DC075018C0181EF9FEF7E
:105DB00050E4A52EB12CB501601B710B7AAB69AB19
:105DC0009C012E193F093EAB2DAB37FF05C0319525
:105DD000219531093EAB2DABC9A8DAA8D7FE03C087
:105DE0003FEFC31AD30AD594C794E816F9060CF00E
:105DF00054C081E0482F880F550B5FAF4EAFA016FF
:105E0000B1060CF44FC06CAD7DAD40E046165706B0
:105E10000CF045C0B801C7010E9467188DA99EA962
:105E2000C81AD90AD7FE08C02EAD3FADE20EF31E48
:105E300049A95AA9C40ED51E0F5F1F4FE0CF0C33DE
:105E4000110509F44ECE9091A3019111E3C6882368
:105E500009F447CE815043CEFFA8FF2009F47FCE3E
:105E600071117DCE1093140100931301B0921601AD
:105E7000A092150174CE40E4E42EF12C01EF1FEF47
:105E80009ACF3A2D2B2D5C01832F922F31EFE32EE9
:105E9000FF24FA9400E410E08ECF8FEFABCFB70170
:105EA000C801BACF8091A201813009F068C086E0B4
:105EB000E7E0F1E0DE01179601900D928A95E1F797
:105EC00040910701509108012091090130910A0188
:105ED00060910B0110910C0186E0E3E1F1E0DE013D
:105EE000119601900D928A95E1F78091130190919E
:105EF0001401640F752F711D86179707DCF5BC011F
:105F0000FBA86F0D711D46175707A4F5A901410F96
:105F1000511D2416350674F5FCA82F0C311C2215D2
:105F2000330544F520919F0121110EC00A969093EC
:105F30001401809313018BEF9FEF909308018093DE
:105F4000070183E080939F0180919F01813091F44C
:105F500080911301909114010A97909314018093FA
:105F6000130181E890E0909308018093070183E09A
:105F700080939F016AAD7BAD672B91F162C02AAD22
:105F80003BAD232B09F05DC0823051F58091A0011B
:105F9000813031F5C30101969093100180930F0178
:105FA0003FEF231A330A309216012092150188AD73
:105FB00099AD01969093200180931F01809121015A
:105FC000909122010196909322018093210180916A
:105FD0002301909124010196909324018093230141
:105FE00080910F0190911001C19759F58FA98150AF
:105FF0008093A10180919E018F5F80939E010E94FA
:10600000B9362EE030E040E050E00E942737609340
:106010009F016111D4C04CE95FEF50930801409398
:10602000070180912801813061F485E08093BD01F2
:1060300080E48093900087E893E1909399008093A7
:1060400098008091A10196EF980F9A3560F4909294
:10605000B8018092B70129E330E03093BA01209370
:10606000B9010E94EF1D8091A101843660F0109269
:10607000B8011092B70129E330E03093BA012093C0
:10608000B9010E94EF1D8091A1018A3070F427E0D0
:1060900030E03093B8012093B70129E330E030932A
:1060A000BA012093B9010E94EF1D8091AC0180FDDF
:1060B00097C040910F015091100141335105C9F42F
:1060C00080919C0190919D01019690939D018093F8
:1060D0009C01809106018A3160F090919E019B3075
:1060E00040F0909105019F5F90930501815080934E
:1060F000060120910D0130910E01809113019091C4
:106100001401B90163507109861797070CF461C037
:106110006A5F7F4F681779070CF45BC04133510504
:1061200009F05EC040919C0150919D014E5F5F4F10
:1061300050939D0140939C012817390709F050C0E6
:1061400080912801813061F485E08093BD0180E475
:106150008093900083EC99E090939900809398004D
:1061600080919B018F5F80939B0180919A018C5E4F
:1061700080939A012091A9013091AA012F5F3F4F8E
:106180003093AA012093A9018B3318F08AE38093FE
:106190009A0180919C0190919D01039690939D019D
:1061A00080939C01809106018733D0F49091050182
:1061B0009350909305018D5F8093060111C061306B
:1061C00009F02FCF60EE70E0709308016093070133
:1061D00028CF2817390721F44133510509F4B0CFEE
:1061E00010919A01112309F443C020E04FE359E0D4
:1061F00070E060E087E190E00E94A01700E022E0FC
:10620000412F62E070E083E290E00E942C1924E0CC
:106210004BE361E070E082E290E00E944E198091D1
:10622000AC019091AD016BE070E00E948A37892B40
:1062300019F4115010939A0180919A018A33C0F099
:1062400080919C0190919D01449690939D01809333
:106250009C01809199018F5F809399018091A801A1
:106260008F5F8093A80110929A0181E0809398013A
:1062700080919C0190919D0123E730E08436910547
:1062800014F02EE630E03093B8012093B70129E3F3
:1062900030E03093BA012093B9010E94541B8091E1
:1062A0009E018B3008F462C0209106018DEC820FB4
:1062B000843018F489E08093040182ED820F8430E9
:1062C00018F486E08093040181EE820F8E3018F47A
:1062D00084E0809304018BEE820F893018F483E010
:1062E000809304016091040170E08091AC01909171
:1062F000AD010E948A37892BC9F580910D019091DB
:106300000E014091050150E0841795071CF031E023
:106310003093970130E0281739070CF481C41092AC
:106320009701841795078CF4019690930E01809342
:106330000D01281739074CF420919701213029F4D9
:10634000019790930E0180930D018091A2018230FC
:1063500069F48091970181118CC080911301909113
:1063600014010196909314018093130180911501FB
:106370009091160180349105D1F4809127018150CC
:10638000809327018091A7018F5F8093A70180915F
:106390002801813061F485E08093BD0180E4809321
:1063A00090008FE19EE490939900809398008091F3
:1063B0002701833009F066C000E023E043E06CE38E
:1063C00070E084E190E00E942C1923E043E068E350
:1063D00070E084E190E00E942C1923E043E064E344
:1063E00070E084E190E00E942C191091B00111300E
:1063F00009F05DC080910301813029F488E1809328
:10640000A101109203010E948A1A0091A10111308A
:1064100009F055C460910F017091100120E043EE26
:1064200058E080910D0190910E010E94D417013027
:1064300069F4209115013091160180911B01909112
:106440001C012817390711F41093960180919601C9
:10645000813009F0C0C0609115017091160120E0F3
:1064600045EA58E080911301909114010E94A01711
:10647000BAC0813009F07ACF809113019091140154
:10648000019770CF823071F400E023E043E068E3CD
:1064900070E084E190E00E942C1923E043E06CE37B
:1064A00070E09FCF813009F0A0CF00E0F6CF12302E
:1064B00039F480910301813009F0A5CF85E29FCFA7
:1064C000133009F0F9C380910301813029F488E386
:1064D0008093A101109203010E948A1A1091A101D8
:1064E00060910F017091100122E043EE58E080911D
:1064F0000D0190910E010E94D417113069F4209182
:1065000015013091160180911B0190911C012817F3
:10651000390711F41093960180919601813009F4A6
:106520009ACF811160C0609115017091160122E02F
:106530003FC210919E011431D0F460911501709109
:10654000160120E043EE58E0809113019091140170
:106550000E94D41760910F017091100120E043EE6A
:1065600058E080910D0190910E010E94D4178CEE9D
:10657000810F8431D8F4609115017091160121E0EA
:1065800043EE58E080911301909114010E94D417BA
:1065900060910F017091100121E043EE58E080916D
:1065A0000D0190910E010E94D4171DC01832D8F031
:1065B000609115017091160122E043EE58E0809140
:1065C0001301909114010E94D41760910F017091F2
:1065D000100122E0E2CF609115017091160120E0D8
:1065E000882309F4E5C18091A1018111EEC0809159
:1065F000AC019091AD01B4010E948A37892B61F4FE
:1066000080910101909102018E3191052CF4019647
:106610009093020180930101009101011091020108
:1066200020E047E058E0B8018DE290E00E94A0171A
:106630000D31110539F480919501811103C081E07C
:106640008093950184E00E945918882339F0809145
:106650009501823019F483E08093950184E00E94D3
:106660005918882339F080919501813019F482E01E
:106670008093950180919501823009F043C000E03C
:106680002DE244E66BE070E08FE090E00E942C1970
:1066900003E110E01093B8010093B7018FE090E0A0
:1066A0009093BA018093B90189EF97E00E94E818AE
:1066B00080919C0190919D010E94541B1093B80100
:1066C0000093B7018EE190E09093BA018093B901F5
:1066D00080EF97E00E94E81880919B010E94EF1DD7
:1066E0001093B8010093B7018DE290E09093BA0146
:1066F0008093B90181EE97E00E94E818809199019A
:106700000E94EF1D80912801813009F05EC08091C8
:1067100001019091020197FF0CC088E08093BD01B8
:1067200080E48093900083EC99E0909399008093AB
:10673000980080910101909102010197029760F405
:1067400083E08093BD0180E4809390002FEC37E0DC
:10675000309399002093980080910101909102015B
:106760000497049760F483E08093BD0180E48093F4
:10677000900082E896E09093990080939800809131
:106780000101909102010997049760F483E08093DE
:10679000BD0180E4809390004FEC57E05093990046
:1067A0004093980080910101909102010E97099702
:1067B00060F488E08093BD0180E48093900061EEF6
:1067C00074E07093990060939800809198018130F3
:1067D00009F041C08091940111E0180F10939401C9
:1067E000143128F08E51833110F0173448F020E036
:1067F0004DE957E06CE170E085E590E00E94D41728
:10680000809128018130F9F4163060F485E080939E
:10681000BD0180E4809390008FEC97E09093990005
:10682000809398008091940186508E3060F483E0CC
:106830008093BD0180E48093900026E534E030939E
:1068400099002093980080919401863921F4109248
:1068500094011092980100919E010B3008F4C8C079
:106860008091AC019091AD0165E070E00E948A37A3
:10687000892B29F4809193018F5F809393018091FC
:106880009301823010F01092930180919F01811149
:1068900096C08091070190910801813891052CF4F0
:1068A000029690930801809307016091090170910D
:1068B0000A012091930147E857E0809107019091E8
:1068C00008010E94A01710919F01143009F0ADC07B
:1068D00020E04FE057E070E060E081E790E00E9448
:1068E000D417093108F4C9C0063208F4C3C088EFD0
:1068F000810F833048F422E04FE057E070E060E021
:1069000081E790E00E94D41785EF810F833008F073
:10691000B1C022E04DEA56E070E060E081E790E02F
:106920000E94D417173009F0C4C08091A2018130B1
:1069300009F0B9C180911501909116018931910535
:1069400039F08C31910521F08D7F819709F0ABC131
:1069500080911301909114010297A1C11091A1019E
:1069600060910F017091100121E043EE58E0809199
:106970000D0190910E010E94D417113069F42091FD
:1069800015013091160180911B0190911C0128176F
:10699000390711F41093960180919601813009F422
:1069A0005ACD609115017091160121E081111BCE25
:1069B00043EE58E08091130190911401F4CD8130A1
:1069C00009F081CF80910701909108018C3F3FEF42
:1069D00093072CF002979093080180930701609130
:1069E000090170910A012091930141E757E065CFB9
:1069F000063008F068CF88E00E945918882319F003
:106A000084E08093D30180E10E945918882319F013
:106A100083E08093D3018091270181110C94FD23A1
:106A200085E08093D3010C94FD23153009F001C15A
:106A300020E04DEA56E070E060E081E790E00E94DF
:106A4000D417093108F050CF8091A201813071F53F
:106A500080911501909116018931910529F08E31AF
:106A6000910511F0839711F5809113019091140114
:106A7000019718C0143009F0F3C08091A201813051
:106A8000A9F480911501909116018931910529F0A1
:106A90008E31910511F0839749F480911301909103
:106AA000140101969093140180931301093108F4A5
:106AB000A2CF063208F49FCF88EF810F8330D0F445
:106AC0008091A2018130B1F480911501909116015D
:106AD0008931910531F08C31910519F08D7F8197C5
:106AE00049F480911301909114010496909314013C
:106AF000809313011B50133008F07DCF8091A201C9
:106B0000813009F078CF809115019091160189317B
:106B1000910539F08C31910521F08D7F819709F035
:106B20006ACF8091130190911401049790931401FE
:106B30008093130160CF82E390E09093B80180933B
:106B4000B7018EE190E09093BA018093B9018CE98E
:106B50009DE10E94E81880E10E945918882311F4F1
:106B60000C94FD2382E05DCF8EE190E09093B8011C
:106B70008093B7018AE090E09093BA018093B901C5
:106B800080E99DE10E94E81889E190E09093B801C6
:106B90008093B7019093BA018093B90182E89DE197
:106BA0000E94E8188BE190E09093B8018093B701C0
:106BB00088E290E09093BA018093B90185E79DE166
:106BC0000E94E8189092B8018092B70107E310E0A4
:106BD0001093BA010093B9018EE69DE10E94E81876
:106BE0008AE590E09093B8018093B7011093BA01C1
:106BF0000093B90187E69DE10E94E81884E00E94B5
:106C00005918882329F00E941C1A81E08093D3012F
:106C100088E0A2CF913011F40C946C2D0C94712D5E
:106C2000841795070CF088CB40919701411184CBD4
:106C30007BCB093108F4DFCE21E04FE057E016307E
:106C400031F0173009F042C021E04DEA56E070E023
:106C500060E081E790E00E94D417063208F054CE3D
:106C6000153009F4F1CE093108F4C5CE163009F01B
:106C700059CE8091A2018130B1F48091150190919B
:106C800016018931910531F08C31910519F08D7F14
:106C9000819749F480911301909114010296909389
:106CA000140180931301063208F024CFA4CE913052
:106CB00009F4CDC80C94712D112309F43ACC12308B
:106CC00009F44CCE133009F409CC8DCC063208F00F
:106CD0000ECE153009F4B8CEC9CF8F929F92AF92E5
:106CE000BF92CF92DF92EF92FF92CF93DF93EC01AE
:106CF000688179818A819B81611571058105910582
:106D000021F464E279ED8BE597E02DE133EF41E08A
:106D100050E00E94273749015A019B01AC01A7EAC4
:106D2000B1E40E9446376B017C01ACEEB4EFA501E3
:106D300094010E945437C60ED71EE81EF91EF7FEB6
:106D400006C081E0C81AD108E10880E8F80AC882C4
:106D5000D982EA82FB82C701B6019F77DF91CF918A
:106D6000FF90EF90DF90CF90BF90AF909F908F906B
:106D700008958F929F92AF92BF92CF92DF92EF923F
:106D8000FF926091360170913701809138019091A6
:106D90003901611571058105910521F464E279EDF0
:106DA0008BE597E02DE133EF41E050E00E9427377B
:106DB00049015A019B01AC01A7EAB1E40E944637A0
:106DC0006B017C01ACEEB4EFA50194010E94543735
:106DD000C60ED71EE81EF91EF7FE06C081E0C81ACF
:106DE000D108E10880E8F80AC0923601D092370154
:106DF000E0923801F0923901C701B6019F77FF9008
:106E0000EF90DF90CF90BF90AF909F908F900895BC
:106E10006093360170933701809338019093390164
:106E20000895F999FECF92BD81BDF89A992780B552
:106E30000895262FF999FECF1FBA92BD81BD20BDBE
:106E40000FB6F894FA9AF99A0FBE01960895052E96
:106E500097FB1EF400940E943E3757FD07D00E9416
:106E6000593707FC03D04EF40C943E3750954095AB
:106E7000309521953F4F4F4F5F4F089590958095E6
:106E8000709561957F4F8F4F9F4F08950E947B377C
:106E9000A59F900DB49F900DA49F800D911D11246E
:106EA0000895B7FF0C9446370E944637821B930B18
:106EB0000895A1E21A2EAA1BBB1BFD010DC0AA1F3B
:106EC000BB1FEE1FFF1FA217B307E407F50720F053
:106ED000A21BB30BE40BF50B661F771F881F991FCE
:106EE0001A9469F760957095809590959B01AC0117
:106EF000BD01CF010895A29FB001B39FC001A39F20
:106F0000700D811D1124911DB29F700D811D1124E2
:106F1000911D0895AA1BBB1B51E107C0AA1FBB1FEF
:106F2000A617B70710F0A61BB70B881F991F5A9515
:106F3000A9F780959095BC01CD010895EE0FFF1F34
:0C6F40000590F491E02D0994F894FFCF27
:106F4C0010F6FF01113A3A9CFF200005053A00307B
:106F5C00000F0F200003000F0F200005000F0FC0C3
:106F6C00FF80FF40FF1501030101FFFFFFFF00E160
:106F7C0000000000000001000000040405050506E7
:106F8C000606070707080808080909090A0A0B0B6F
:106F9C000B0C0C0C0C00C1808100000000000000E8
:106FAC009A133215BB13B0130114BF13DD13000079
:106FBC0000008518AD14031B021B2F003133000099
:00000001FF
